:020000020000FC
:047000000C948D3E21
:047028000C94B73DD0
:10702F0012010002FF010020EB03F42F0000010208
:10703F00030109021200010100803209040000005F
:10704F00000000000C03410054004D0045004C00AF
:10705F001603410054006D00330032005500340018
:10706F004400460055000C0331002E0030002E0066
:10707F0030000403090416010C0100000C0000018C
:02708F006C7F14
:1070920012BD01BDF89A00B5089501E00895F9996D
:1070A200FECF12BD01BD20BDFA9AF99AF6CFF99929
:1070B200FECF0C944938F80104910895F8013491F7
:1070C20031962491890108950091610000930C0189
:1070D20000E80093610001E00093610005BF02E057
:1070E20005BF0C9486380091D70001600093D70049
:1070F200A89507EF04BF0091600000610093600053
:1071020000E00093600001E008950E94AA3D0E9401
:10711200B53DFDCF0CD00F7708D0006806D00061D6
:1071220004D0016028D0789408950093D80000918B
:10713200D8000895FCDF00621ED04CD009B500FFD4
:10714200FDCFF5DF0F7D17D00091E0000E7F009399
:10715200E0000091E000077F0093E0000091E20070
:1071620001600093E2000091E20008600093E200F7
:1071720078940C94743B0093D800089500910D010B
:10718200002359F40091D90000FF07C0D0DF006846
:10719200F2DF01E000930D01CDDFE0E2F2E00081D9
:1071A200018100FF0DC0008111811E7F11830083C8
:1071B20001E00093EA0000E00093EA0000931E025F
:1071C20000E00093E9000091E80003FF02C00E9482
:1071D200F23B0895A89539D000E40093600000E0E6
:1071E200009381000093800010E0009385000093DB
:1071F200840001E006BB00918100036000938100DE
:107202000091600007FFFCCF00E80093600010933C
:107212008100A89507EF04BF18D010936000209159
:1072220084003091850010938100109380001093A8
:1072320085001093840001E006BB2D3D354010F01F
:1072420002E101C002E009BD089500916000006101
:107252000093600008950E94AD3E239741D100E063
:1072620000930901B5D104811581012B51F437D165
:1072720000910701002309F4B9C000E0009307015F
:10728200B5C058D102FFFDCF37D1068335D1009367
:107292000F0132D1009310012FD1009311012CD193
:1072A2000093120129D10093130102852091130149
:1072B20030911201409111015091100116811A95DD
:1072C20041F01250A9F01A9599F11A9509F473C078
:1072D2008BC010910F01113011F411E001C010E0C8
:1072E200138799D00C3F11F414D17FC077D17DC0A0
:1072F20092D010910F01112329F01A9549F01A9595
:10730200A9F073C010E013870C3F09F06EC0ECCFF8
:1073120056D103C04CD109F468C00D911C9144D1DF
:107322000F3FC1F305E0009309015FC011E0EBCF0D
:10733200D2D029F00250E1F10A9541F056C0FDD0B9
:107342000E94A33F0FEF00930A014FC0552319F08B
:107352005A9579F04AC04ED00DEF04BF74D0EAD0EE
:1073620003FFFDCF67D051D04AD008E00093600000
:10737200FFCF40D068D0DED003FFFDCF5BD03FD03F
:1073820044D00FEF1FE004C009811A810150104060
:1073920009831A8309811A81012BB1F700E800934E
:1073A200610000910C01009361000C940000FFCF7A
:1073B20001E003871AC08FD019F00A9539F015C081
:1073C200535098F4BAD002E000870FC0505339F0FE
:1073D2005A9541F05F52B1F35A95A1F306C002E00B
:1073E2000883F0CF01E0FCCFA8D079D02396E4E067
:1073F2000C94BA3E01E005BF00E005BF089500917C
:10740200D8000F770093D800089509B50D7F09BD04
:1074120000E009BD08955183408333832283109194
:10742200E8001B7F1093E8001091E8001F7710938B
:10743200E80008955DD053D0F8940091E000016017
:107442000093E000089579D04AC0219749D0009175
:107452000601035019F00250B9F00BC03CD021F0E4
:107462000A9559F00A9529F400910A010C3F19F482
:1074720050D02196089567D0FCCF0091010100936E
:10748200F100009100010AC01091100124D019F0FE
:107492000A9549F0EECF135018F400E00093F10082
:1074A2001ED044D0E6CF105339F01A9539F01F524E
:1074B20041F01A9541F0F4CF08E5F0CF00E006D094
:1074C200EDCF02E0FCCF04E001D0E8CF10E020E0F5
:1074D20030E00C94113F00910F010023089521C068
:1074E2000BD008D007D00093040106D00093050109
:1074F20021D00BC000D008830091F10008950091C3
:10750200EB0000620093EB0015D0077F0093E800C8
:107512000895F5DF02E00093080103E000930901FA
:10752200089559D007D000FFFDCF089503D002FF80
:10753200FDCF03C00091E8000895FCDF0B7FE6DF7A
:10754200F9DF0F77E3CF0E94AC3E42D038D006C0BD
:107552002BD00093F1002BD059F43DD0082F092BEA
:10756200A9F0E8DF02FD12C0E5DF00FFFDCF4424F1
:10757200042D4394003289F300910B0100230D91F5
:107582001C9131F311970E945838E3CFD3DF00FFEB
:10759200FDCF21D0CFDF00FFFDCFCCDF02FFFDCF3B
:1075A200CCDFE5E00C94B93E11970C945C380D9158
:1075B2001C910F5F1F4F1C930E93019708958281B8
:1075C200938100811181801B910B0196DF01089547
:1075D200E0E0F1E00895AEDF0E7F98CF0E94A93E71
:1075E200F7DF80819181A081B181AF710481158122
:1075F20000521040048315830AC000910B0100233E
:1076020031F4A301920103E911E00E943B3F47D00C
:10761200B8F1662477242C0111C06EDFF301ED5618
:10762200FE4F008301E0600E00E0701E01960091A3
:10763200F200002311F033D0B8F47FDF30D0E8F24B
:10764200F301B096E238F040C0F674DF02FFFDCFDE
:107652000091F200BDDF24813581201B304024835C
:107662003583E5CF49DFAA95AA23E1F700910B0103
:10767200013099F62091F1008C010E945038D6CF4A
:1076820004811581012B21F055DF02FFFDCF55DF6B
:10769200A2DF50DF00FFFDCFE8E00C94B63EE0E051
:1076A200F1E0028113810817190708952091EB0078
:1076B20021602093EB000093EC000091ED0002703A
:1076C200012B0093ED000091ED0002600093ED00AC
:1076D2001091EE00012F000F00E0001F0895412FCE
:1076E2000093E900089500E009D000FD05C000E024
:1076F200F7DF10E202E0DACF00E00895F1DF009157
:10770200EB0008950F770132A9F5112369F11A955B
:1077120059F01A9561F01A9569F01A95F9F01A95CF
:10772200C1F01A95D9F024C00E942C3920C00E94C1
:10773200263A1DC029D00091090123D001E01FD0B3
:1077420020D0009108011BD00E94923A0E94973AE1
:107752000EC01AD00091080114D007C002E00093B5
:10776200080100E0009309010FD00E94923A03C081
:107772000E94803A02C001E0089500E0089501D01D
:1077820000E00093F10008950091E800077F009364
:10779200E800089508950350F9F4112339F01A9579
:1077A20051F01A9581F01A9599F016C004E016D09E
:1077B20001E810E703C011D003E510E7E7E1F2E0CA
:1077C20000831183D8CF06E109D00FE510E7F6CF89
:1077D20004D005E710E7F2CFD0CF0CE000931A02F5
:1077E200089527D120D100931D02E1D0212F11232A
:1077F20029F12A95E9F02250F1F0225099F02A95C8
:1078020049F0225061F02A9581F02A95E1F02A95FB
:10781200E9F023C0003809F44FC00C94833B0038D0
:10782200E1F7C8C00023C9F71EC00023B1F72DC07D
:10783200033098F744C1033080F70BC1003868F376
:10784200033858F7C9C0013841F77BC1013051F400
:10785200FCD0BFD000FD06C0FCCF0E94833B0023BA
:1078620009F41ED008951091E3001078DCD00F7750
:10787200012B0093E300E9D0ACD000FFFDCF0091D3
:10788200E30000680093E300089591D0123040F4C1
:107892000FD010931E02DAD000911E020C94CB3B43
:1078A2000091EB0001D004C000620093EB00089548
:1078B2000091E800077FC0C0BA93AA93229700E024
:1078C2000093190274D0AFD0202F2A9519F02A956F
:1078D200E9F022C002E100931A020FE210E7E7E1A9
:1078E200F2E0008311839DD008839DD00983E0DFFD
:1078F20000911A0210E02881398102171307A8F4B7
:107902000F7181F401E00093190211C002E10093AA
:107912001A0201E410E7E3CF0E94CC3B002319F7DF
:107922008ED040C01093190202C020931A027ED05A
:10793200A7E1B2E001C08AD000911A02002309F146
:1079420048D004FD1EC045D000FD03C042D004FF54
:10795200FACF10E0012F1395003281F0ED91FC91E6
:107962001197049133D02D913C912F5F3F4F3C935F
:107972002E93FD0103810A95038361F72AD004FF48
:10798200DACF00911902013039F423D004FD04C08A
:1079920020D000FFFDCF5AD01CD004FFFDCF46D02F
:1079A20018D00B7F49D02296A991B99108951091D0
:1079B200F10008957DDF00911E0208D047D009D062
:1079C2000F773AD006D002FFFDCFBFC00093F1007F
:1079D20008950091E800089524D010911D021058D6
:1079E20029F01A9589F01A9591F019C061DF00917A
:1079F2001C02ECDF00E0EADF29D0EBDF02FFFDCF63
:107A020018D0E7DF0F770CC053DF00E0F2CF51D080
:107A12000F7710E0F801E55EFD4F0081EACF0FD04D
:107A22000BC001D000D00091F1000895D2DF0F7E8B
:107A320003C00091E8000B7F0093E80008950091D5
:107A4200EB0032DFC6DF077F089532DFC2DF0E7F31
:107A5200F3CF00911D02002329F00A9509F10A953E
:107A620031F01EC0E0DF0A9561D0D9F41AC061D0AE
:107A7200B9F4D9DF0F7711F416D01BD00093E900C7
:107A82001091EB0010FF0BC00ED010E01093E90034
:107A920021E0F801E55EFD4F20834FD003C042D0C4
:107AA20045D0CFDFC9CF1091EB0010621093EB00ED
:107AB20008951091E800177F1093E800089500914F
:107AC2001D02002311F4AFDF02C0013011F4B7DF51
:107AD200B3CF023031F52DD019F52091F1002F7777
:107AE2002093E90023D000FF19C081F01FD000616C
:107AF200DCDE01E010E0422F0E949F3E0093EA008C
:107B020000E00093EA0012D00860CFDE0BD030E034
:107B1200F901E55EFD4F008310D0DACF03D0D7CF55
:107B2200BFDE089500E00093E90008950091EB00A4
:107B3200089579DF3CDF00230895BADE4ADF0E7F25
:107B4200089583DF46DF02FFFDCF73DF42DF0F7749
:107B520073CF0091D70001600093D7000E948B3849
:107B620000E000931F0208950C94BF388A93FA93A1
:107B7200EA933A922A921A920A927A936A935A93BF
:107B82004A933A932A931A930A938FB70091DA0091
:107B920000FF24C00091D80000FF20C00EEF009328
:107BA200DA000091D90000FF11C001E000930D013D
:107BB200ABD0026096D09AD00860A2D00E949B38C7
:107BC2000091E0000E7F0093E00008C000E0009307
:107BD2000D0100931E0298D0046083D07FD002FF73
:107BE20005C084D002FF02C00BEF75D077D000FF32
:107BF2001BC07CD000FF18C001E000930E016AD0C8
:107C020083D000626ED00EEF6FD0006179D06ED05B
:107C12000F7D76D00091D80000620093D80009B59C
:107C22000D7F09BD00E009BD59D004FF20C05ED020
:107C320004FF1DC009B500FD05C00E94EB3809B55F
:107C420000FFFDCF0091D8000F7D0093D80042D0F5
:107C520000910E01002359F04CD00FEE45D00F7E5B
:107C620052D000643ED042D001604AD042D036D0D9
:107C720005FF0FC03BD005FF0CC000E000930E01D2
:107C820035D00F7E3DD00FED2FD00F7D3CD0006858
:107C920028D024D003FF0DC029D003FF0AC000E082
:107CA20000931F0207EF17D00E94743B2DD0116082
:107CB20018D08FBF09911991299139914991599100
:107CC200699179910990199029903990E991F991E6
:107CD200899118950FEE0093E10008950091E1005B
:107CE20008951183008308950093E1000091E2005A
:107CF20008950091E200006203D00091E200086062
:107D02000093E2000895FCDFE0E2F2E000811181DD
:107D1200089500008895FECF01E60DBF02E00EBF78
:107D2200C2EED2E00E947438002311F00E94D33ECA
:107D32000E9465380E948A3E0C948A3E4A951AF047
:107D4200000F111FFBCF0895BA92AA929A928A92BB
:107D52007A926A925A924A92BA93AA939A938A937D
:107D62000895BB84AA84998488847F806E805D8014
:107D72004C80BB81AA8199818881F0E00FB6F8948A
:107D8200CE0FDF1F0FBE089520E006D0E9F7089559
:107D9200259102D0E9F708952D9301501040202F2C
:107DA200212B089585E890E7FC0105911491FC01CF
:107DB2003296A591B491FC01349625913491422FCB
:107DC200432B19F0F901E4DF01C0DEDF069610E76C
:107DD2008139910748F308952F930CD02F9101D048
:107DE20008953CD0F12FE02F45E047BFE89536D00B
:107DF20012D0089533D0F12FE02F43E047BFE8952A
:107E02002DD008952BD0F12FE02F43E047BFE89506
:107E120025D001D0089522D041E147BFE8951EC088
:107E22001DD0F12FE02F41E247BFC895002D16C0AB
:107E320015D0F12FE02F49E047BFC895002D0EC0A5
:107E4200F32FE22F012E102E41E047BFE89506C026
:107E520005D0002E29E027BFE89500C0022E27B7E3
:107E620020FDFCCF202D0895022E27B726FDFCCF42
:107E7200202D08950E94A53E22974801C901DA01EA
:107E820010C05BD001E0A00E00E0B01E00E4A0161E
:107E920000E0B00608F440C0830120E030E00E9418
:107EA200F23E0A2F0B2B09F440C0082F0F7710E087
:107EB2002C01401A510A320100E4A02E03C00A2FFD
:107EC2000B2BE1F04816590680F0F40101914F01A5
:107ED2000983119729F001914F010883119711C06D
:107EE200F2013196049108830CC0F20104910983D6
:107EF2003196E817F907A1F7F401EDCF1BD00883FB
:107F020019839201088119810E94213F16D0AA94F7
:107F1200B1F62301AA24BB240DD0312F0F3F3F4FCE
:107F220009F4AFCF83011DD0B7CF01E02296ECE078
:107F32000C94B23E82010C945F3802E0400E00E0E5
:107F4200501E08959A938A9380E090E08C0109D0A4
:107F520080589F4F8F3F0FE69007C0F38991999108
:107F6200089520E030E00C94FB3E00000000000089
:067F720000000000FC000D
:107FE4000C94ED3E0C94113F0C94193F0C94213FDA
:0C7FF4000C94F23E0C94033F0C94293FC7
:040000030000700089
:100000000C94A0050C94E4050C94E4050C94E40510
:100010000C94E4050C94E4050C94E4050C94E405BC
:100020000C94E4050C94E4050C94B6180C9488190F
:100030000C94A1270C94E4050C94E4050C94E405BD
:100040000C94E4050C94E4050C94E4050C94E4058C
:100050000C94E4050C9409280C94E4050C94E40534
:100060000C94E4050C94E4050C94E4050C94E4056C
:100070000C94E4050C94E4050C94E4050C94E4055C
:100080000C94090F0C94E4050C94E4050C94E4051D
:100090000C94E4050C94E4050C94E4050C94E4053C
:1000A0000C94E4050C94E4050C94E4053F064F061B
:1000B000610671067706860692069706A406AC06C8
:1000C000BC06C106C813C813C813C813C813C81385
:1000D000C813C813C813C813DF13DF13DF13DF13EC
:1000E000DF13DF13DF13DF13DF13DF13C813C813AE
:1000F000C813C813C813DF13DF13DF13DF13DF13B5
:10010000C813C813C813DF13DF13DF13F519171A49
:10011000051B171A051B5C1A7F1A051BD41AE71A50
:10012000EA1DEA1D271E271E811EBF1E372137210B
:10013000D81E3721D91FD91F9C20B3203721222157
:1001400007634236B79BD8A71A39685618AEBAABC0
:10015000558C1D3CB7CC5763BD6DEDFD753EF61754
:100160007231BF000000803F08000000BE922449A9
:10017000123EABAAAA2ABECDCCCC4C3E00000080D9
:10018000BEABAAAAAA3E00000000BF000000803F4C
:100190000000000000084178D3BB4387D1133D190C
:1001A0000E3CC3BD4282AD2B3E68EC8276BED98F39
:1001B000E1A93E4C80EFFFBE01C4FF7F3F0000007D
:1001C000000035001E001F00200021002200230037
:1001D00024002500260027002A002B0014001A0006
:1001E0000800150017001C0018000C001200130076
:1001F0004C00290004001600070009000A000B004B
:100200000D000E000F0033003400E1001D001B0044
:1002100006001900050011001000360037003800F4
:1002200028000530E000E200E30003302C002C0041
:1002300004305000510052004F0035001E001F00D6
:100240002000210022002300240025002600270092
:100250002A002B0014001A00090013000A000D00E8
:100260000F0018001C0033004C002900040015008A
:100270001600170007000B00110008000C00120008
:100280003400E1001D001B000600190005000E00EF
:10029000100036003700380028000530E000E2008A
:1002A000E30003302C002C000430500051005200B9
:1002B0004F0035001E001F002000210022002300F7
:1002C00024002500260027002A002B0034003600D9
:1002D000370013001C0009000A00060015000F007B
:1002E0004C00290004001200080018000C00070050
:1002F0000B001700110016003800E1003300140055
:100300000D000E001B00050010001A0019001D0052
:1003100028000530E000E200E30003302C002C0050
:1003200004305000510052004F0035021E021F02DF
:100330002002210222022302240225022602270291
:100340002A0035021E021F0220022102220223027D
:1003500024022502260227024C004C003A003B00F2
:100360003C003D003E003F002D022E022F023002D5
:1003700031020100400041004200430044004500BA
:100380000100010001000100010001000100010065
:1003900001000100010001000100AB00AA00A9005A
:1003A000AE0035001E001F002000210022002300A7
:1003B00024002500260027002A0035001E001F000B
:1003C0002000210022002300240025002600270011
:1003D0004C004C003A003B003C003D003E003F001A
:1003E0002D002E002F0030003100010040004100A0
:1003F00042004300440045000100010001000100EB
:1004000001000100010001000100010001000100E4
:100410000100AB00AA00A900AE000000000000002F
:1004200000000000000000000000000000000000CC
:1004300000000000000000000000000000000000BC
:1004400000000000000000000000000000000000AC
:10045000000000000000000000000000000000009C
:10046000000000000000000000000000000000008C
:10047000000000000000000000000000000000007C
:100480000000033000000000043000000000000005
:10049000000000000000000000000000000000005C
:1004A000000000000000000000000000000000004C
:1004B000000000000000000000000000000000003C
:1004C000000000000000000000000000000000002C
:1009400000003A003B003C003D003E003F004000FC
:1009500041004200430044004500010000500100F6
:10096000010001000100010001000100010001007F
:100970004C000100010001000730063013501250F6
:100980000030013002300100010001000B300A305C
:1009900009300830010001000100010001000100E0
:1009A000010001000100010001000100010001003F
:1009B000010001000100010001002A035400680049
:1009C000650020005000720065006F006E00690035
:1009D000630020004B006500790062006F00610039
:1009E0007200640000002C034F0072007400680065
:1009F0006F006C0069006E006500610072002000ED
:100A00004B006500790062006F00610072006400B5
:100A1000730000000403090409025400030100A04C
:100A2000FA0904000001030101000921110100017C
:100A3000223F000705810308000A090401000103A1
:100A4000010200092111010001224D000705820366
:100A500008000A0904020001030000000921110135
:100A600000012236000705830308000A1201100165
:100A700000000008EDFE61600100010200010501B7
:100A80000980A101850216010026B7001A01002A7B
:100A9000B700751095018100C0050C0901A1018501
:100AA00003160100269C021A01002A9C027510956B
:100AB000018100C005010902A1010901A100050988
:100AC000190129051500250195057501810295017A
:100AD000750381010501093009311581257F9502D2
:100AE0007508810609381581257F950175088106ED
:100AF000050C0A38021581257F950175088106C00D
:100B0000C005010906A101050719E029E71500251F
:100B10000195087501810295017508810105081983
:100B2000012905950575019102950175039101054E
:100B300007190029FF150025FF950675088100C0DB
:100B400011241FBECFEFDAE0DEBFCDBF04B603FE37
:100B500024C08091A3039091A403A091A503B09118
:100B6000A6038730904BA740B04BB9F41092A30373
:100B70001092A4031092A5031092A60314BE84B78A
:100B8000877F84BF88E10FB6F8948093600010924D
:100B900060000FBEE0E0F8E3099512E0A0E0B1E0EC
:100BA000EAEEF2E602C005900D92A83AB107D9F735
:100BB00013E0A8EAB2E001C01D92A33AB107E1F741
:100BC0000E94FC150C9473310C940000279A2F9806
:100BD0008FEF9FEF90938700809386008AE0809349
:100BE000800089E1809381000C94F82C282F8111DA
:100BF0000BC080918000877F8093800010928D00D1
:100C000010928C002F9808952F9880918000886012
:100C100080938000233019F48FEF9FEF0FC083E0A3
:100C200090E0821B9109880F991F2FEF3FEFA901D8
:100C300002C0569547958A95E2F7CA0190938D00B8
:100C400080938C000895CF93DF93EC010E949D2840
:100C5000BE0180E090E0DF91CF910C9417250F93B7
:100C60001F93462F50E04C30510508F098C0DC012E
:100C7000FA01EA5AFF4F12968C910C94373188236F
:100C800009F48DC000E010E0980140E064E070E0FD
:100C90008BEC91E00E94871281E090E00FC08823E6
:100CA00009F47DC000E010E0980140E066E070E0EB
:100CB0008BE591E00E94871282E090E00E9423067B
:100CC0006EC0882309F46BC000E010E0980140E09A
:100CD00068E070E08BE891E00E94871284E090E089
:100CE000EDCF882311F083E005C083E00CC088239A
:100CF00049F084E00E94942540E164E083E00E9492
:100D0000ED0A4DC084E00E94B525F6CF882331F06E
:100D100085EE0E947E1C0E944F2D41C085EE0E94F0
:100D2000461D3DC08823D9F10E941B0E38C0882380
:100D3000B1F10E94140E00E010E0980140E064E080
:100D400070E08BEE91E029C0882349F185E00E9494
:100D5000B5250E943C0E23C0882309F100E010E075
:100D6000980140E068E070E08BE191E00E9487121A
:100D700085E00E94942513C0882389F00E941A13ED
:100D800004C0882361F00E94251300E010E0980160
:100D900040E068E070E08BE191E00E94871280E023
:100DA00090E01F910F9108950F931F932FEF89EFFC
:100DB00090E0215080409040E1F700C0000000E04A
:100DC00010E0980140E064E070E08BEE91E00E945A
:100DD00087121F910F910895CF92DF92EF92FF92A9
:100DE0000F931F93CF93DF93CDB7DEB7CC58D109C4
:100DF0000FB6F894DEBF0FBECDBF2091630325FF71
:100E0000C5C08C01FC01928180910201992309F4F3
:100E100060C096E4E7E2F2E0DE01A95BBF4F01901B
:100E20000D929A95E1F7F8019081E0910001F0911F
:100E30000101E90FF11DEE0FFF1F27E430E02C0F39
:100E40003D1FE20FF31F60817181680F711D8827BC
:100E500077FD8095982F0E94932E20E030E040E4AB
:100E600051E40E94F82D6B017C01F801218185E09D
:100E700090E0821B9109BC01882777FD8095982F0F
:100E80000E94932E9B01AC01C701B6010E94902DD8
:100E90009B01AC0160E070E080E090E40E94AA2F2A
:100EA00020E030E04CE551E40E94472F4FE050E055
:100EB000C457DF4F0FB6F894DEBF0FBECDBFDF9132
:100EC000CF911F910F91FF90EF90DF90CF900C94F6
:100ED000271296E4E7E2F2E0DE01119601900D920E
:100EE0009A95E1F7F8019081E0910001F0910101FC
:100EF000E90FF11DEE0FFF1F21E030E02C0F3D1F29
:100F0000E20FF31F60817181680F711D882777FDE3
:100F10008095982F0E94932E20E030E040E451E429
:100F20000E94F82D6B017C01F801218185E090E0A1
:100F3000821B9109BC01882777FD8095982F0E941C
:100F4000932E9B01AC01C701B6010E94902D9B011D
:100F5000AC0160E070E080E090E40E94AA2F20E005
:100F600030E04CE551E40E94472FC457DF4F0FB6E5
:100F7000F894DEBF0FBECDBFDF91CF911F910F91CF
:100F8000FF90EF90DF90CF900C946F0EC457DF4F1F
:100F90000FB6F894DEBF0FBECDBFDF91CF911F918A
:100FA0000F91FF90EF90DF90CF9008950F931F93D4
:100FB00000E010E0980140E063E070E083E091E041
:100FC0000E9487122FEF82E597E0215080409040E9
:100FD000E1F700C000001F910F91089508950E944D
:100FE000E6056E9A769A0C94D4060C94EE070C944F
:100FF000EC060895880F991FFC01EE5BFF4F859169
:1010000094910895880F991FFC01EE53FE4F85912E
:10101000949108950F931F93CF93DF93EC01811563
:1010200020E49207A0F5C11580E3D80708F0E1C0DD
:10103000C83ED105D8F4C03ED10508F0EEC1C83A8B
:10104000D10578F4C53AD10508F074C0C130D10596
:1010500009F46DC008F4DEC1C430D10508F0DDC16B
:10106000D9C1CB3BD10508F470C0D4C1C11590E201
:10107000D90708F0B9C0C11521E0D20708F0CDC1E9
:10108000C03FD10508F4C6C18E01106506C2C1304B
:1010900080E5D80709F4BDC068F5C13120E4D20766
:1010A00009F4AEC050F4C03190E4D90708F0A5C0EF
:1010B000CF70DD278E01146DF0C1C33120E4D2075B
:1010C00009F4A4C008F49FC0C115D04509F0A2C11D
:1010D0000E945B210E943C0E0E94D6079FEF24E3F2
:1010E0008CE0915020408040E1F700C000000E9459
:1010F0002E28D3C1C11520E6D20730F4C11581E5F1
:10110000D80708F48CC02DC1C11590E7D90708F4A1
:1011100081C1C11520E8D20708F478C1C11580E962
:10112000D80708F077C1DF708E01106AB6C101E000
:1011300010E0B3C1C53AD10509F471C1C63AD10571
:1011400009F070C102E810E4A8C1C83AD10509F459
:101150006CC1C93AD10509F46BC1CA3AD10509F489
:101160006AC1CB3AD10509F469C1CC3AD10509F479
:1011700068C1CD3AD10509F467C1C03BD10509F476
:1011800066C1CE3AD10509F465C1CF3AD10509F45B
:1011900064C1C13BD10509F463C1C23BD10509F467
:1011A00062C1C33BD10509F461C1C43BD10509F457
:1011B00060C1C53BD10509F45FC1C63BD10509F447
:1011C0005EC1C73BD10509F45DC1C83BD10509F437
:1011D0005CC1C93BD10509F45BC1CA3BD10509F427
:1011E0005AC100E014E459C1CE019F700E94020868
:1011F00055C1DD278E01106C50C100E011ED4DC1CD
:1012000000E010ED4AC100E012ED47C100E013ED2F
:1012100044C1809177038160809377033EC10E942F
:101220008A28811102C00E9466280E94A22890E0AC
:101230009093A2038093A103C23090E5D90721F4D3
:101240008091A103816086C0C43020E5D20721F4DB
:101250008091A10382607EC0C63080E5D80721F46A
:101260008091A103846076C0C83090E5D90719F455
:101270008091A10327C0CA3020E5D20721F48091D4
:10128000A103806167C0CC3080E5D80721F480914C
:10129000A10380625FC0CE3090E5D90721F4809130
:1012A000A103806457C0C03120E5D20721F48091AA
:1012B000A10380684FC0C23180E5D80729F480912E
:1012C000A1038460886046C0C33090E5D90721F44B
:1012D0008091A1038E7F3EC0C53020E5D20721F466
:1012E0008091A1038D7F36C0C73080E5D80721F4F7
:1012F0008091A1038B7F2EC0C93090E5D90719F4E6
:101300008091A10326C0CB3020E5D20721F4809143
:10131000A1038F7E1FC0CD3080E5D80721F48091D6
:10132000A1038F7D17C0CF3090E5D90721F48091BC
:10133000A1038F7B0FC0C13120E5D20721F480913A
:10134000A1038F7707C0C331D04531F48091A10349
:101350008B7F877F8093A1038091A1030E94A628A1
:101360009CC08D2F99278F70992781309105D9F4D2
:101370009E012370332702C0880F991F2A95E2F738
:101380009C688E0144E0000F111F4A95E1F7002789
:101390001370802B912B53E0CC0FDD1F5A95E1F792
:1013A000C076DD272FC08230910531F4DC2FCC27A9
:1013B0008E01016F106A71C08330910569F4CE010E
:1013C0008370992701E010E002C0000F111F8A9579
:1013D000E2F7C8019C680FC0049709F05EC0CE0117
:1013E0008370992701E010E002C0000F111F8A9559
:1013F000E2F7C8019A6823E0CC0FDD1F2A95E1F7D8
:10140000C07ED7708C010C2B1D2B47C0DF708E0166
:10141000106243C000E010E040C08E013EC001E811
:1014200010E43BC003E810E438C002EE14E435C019
:1014300009EE14E432C00AEE14E42FC005EB14E404
:101440002CC006EB14E429C007EB14E426C00CEC16
:1014500014E423C00DEC14E420C003E815E41DC01F
:101460000AE815E41AC002E915E417C004E915E416
:1014700014C001E216E411C003E216E40EC004E257
:1014800016E40BC005E216E408C006E216E405C047
:1014900007E216E402C00AE216E4C801DF91CF9128
:1014A0001F910F9108959CE0799FF00111249CE316
:1014B000899FE00DF11D1124E60FF11DEE0FFF1FB6
:1014C000EE53FE4F85919491803E9105E0F4803C6F
:1014D000910558F58133910509F46FC048F48932BC
:1014E000910509F463C08A32910509F46DC072C098
:1014F00089339105E9F082389105D1F08533910562
:1015000009F44DC067C0833E910581F138F4803EF7
:101510009105B9F0823E9105D9F05CC0863E9105F7
:1015200061F1873E9105A1F155C00E94FA07089527
:101530002091A10320FD02C021FF4CC080EE90E06D
:1015400049C08091A10380FFF9CF89E390E042C0B8
:101550008091A10382FF0EC08091A10384FF03C08C
:1015600080E090E037C083EE90E034C08091A1032A
:1015700082FFF2CF82EE90E02DC08091A10383FF25
:101580000BC08091A10384FDEBCF87EE90E022C0D9
:101590008091A10383FFF5CF86EE90E01BC0809180
:1015A000A10385FF07C089E290E014C08091A103E8
:1015B00085FFF9CF85E390E00DC08091A10386FF00
:1015C00007C08AE290E006C08091A10386FFF9CFB0
:1015D00081E390E00E940A080895CF92DF92EF9293
:1015E000FF920F931F9301E010E020E030E06801CC
:1015F000790104C0CC0CDD1CEE1CFF1C8A95D2F7CF
:1016000004C0000F111F221F331F6A95D2F70C2947
:101610001D292E293F29C0906303D0906403E090D8
:101620006503F0906603C022D122E222F322842FC8
:10163000C016D106E206F30641F41F910F91FF9008
:10164000EF90DF90CF900C9494251F910F91FF9015
:10165000EF90DF90CF900C94B52508950C942D0B4E
:101660005F926F927F928F929F92AF92BF92CF9232
:10167000DF92EF92FF920F931F93CF93DF93CDB73B
:10168000DEB72A970FB6F894DEBF0FBECDBFCE01EE
:1016900001966C014E019BE0890E911C20E030E028
:1016A00040E050E060E070E000E010E0E12CF12C60
:1016B0006C2C5D2C8AE0782EAA24A394B12CEDE644
:1016C000F2E0A62DB52D872D01900D928A95E1F7B8
:1016D000F601819191916F01FC01E07FFF27E032DB
:1016E000F10559F48F709927F50102C0EE0FFF1F25
:1016F0008A95E2F7EE2AFF2A37C0E033F10559F464
:101700008F709927F50102C0EE0FFF1F8A95E2F74F
:101710000E2B1F2B29C0E034F10559F48F70992747
:10172000F50102C0EE0FFF1F8A95E2F76E2B7F2BAB
:101730001BC0E035F10559F48F709927F50102C0FF
:10174000EE0FFF1F8A95E2F74E2B5F2B0DC0E036A0
:10175000F10551F48F709927F50102C0EE0FFF1FBC
:101760008A95E2F72E2B3F2BC814D90409F0A7CF96
:1017700084B19E2D9095892384B985B1E82AE5B876
:1017800087B1902F9095892387B988B1082B08B924
:101790008AB1962F909589238AB98BB1682B6BB942
:1017A0008DB1942F909589238DB98EB1482B4EB968
:1017B00080B3922F9095892380BB81B3282B21BBC6
:1017C0002A960FB6F894DEBF0FBECDBFDF91CF9142
:1017D0001F910F91FF90EF90DF90CF90BF90AF904F
:1017E0009F908F907F906F905F9008955F926F921F
:1017F0007F928F929F92AF92BF92CF92DF92EF92A1
:10180000FF920F931F93CF93DF93CDB7DEB7689707
:101810000FB6F894DEBF0FBECDBF85B7806885BF19
:1018200085B7806885BF0E94300BCE0101966C01A0
:101830004E0199E1890E911C20E030E040E050E03B
:1018400060E070E000E010E0E12CF12C6C2C5D2CED
:1018500088E1782EAA24A394B12CE7E7F2E0A62D24
:10186000B52D872D01900D928A95E1F7F6018191B2
:1018700091916F01FC01E07FFF27E032F10559F4FF
:101880008F709927F50102C0EE0FFF1F8A95E2F7CE
:10189000EE2AFF2A37C0E033F10559F48F709927FB
:1018A000F50102C0EE0FFF1F8A95E2F70E2B1F2BEA
:1018B00029C0E034F10559F48F709927F50102C071
:1018C000EE0FFF1F8A95E2F76E2B7F2B1BC0E035D2
:1018D000F10559F48F709927F50102C0EE0FFF1F33
:1018E0008A95E2F74E2B5F2B0DC0E036F10551F4DF
:1018F0008F709927F50102C0EE0FFF1F8A95E2F75E
:101900002E2B3F2BC814D90409F0A7CF84B19E2DEC
:101910009095892384B985B1E82AE5B887B1902FDD
:101920009095892387B988B1082B08B98AB1962F79
:10193000909589238AB98BB1682B6BB98DB1942F9F
:10194000909589238DB98EB1482B4EB980B3922FD3
:101950009095892380BB81B3282B21BBE2EBF2E079
:10196000A8EAB2E0119211921D921D9282E0EC3B26
:10197000F807C1F768960FB6F894DEBF0FBECDBF6B
:10198000DF91CF911F910F91FF90EF90DF90CF905B
:10199000BF90AF909F908F907F906F905F900C94CE
:1019A000EF075F926F927F928F929F92AF92BF925A
:1019B000CF92DF92EF92FF920F931F93CF93DF931B
:1019C000CDB7DEB7A2970FB6F894DEBF0FBECDBF7E
:1019D0006E0149E1C40ED11C88EAA82E82E0B82E1F
:1019E00075019AE0592E460101E010E028E1622ECF
:1019F00035E0732EEDE6F2E0D401852D01900D92D5
:101A00008A95E1F7D6018D919D916D019C01207F12
:101A100033272032310591F424B18F709927F801D2
:101A200002C0EE0FFF1F8A95E2F7CF01922F982B8D
:101A300094B995B18095892385B953C02033310578
:101A400091F427B18F709927A80102C0440F551F48
:101A50008A95E2F7CA01922F982B97B998B1809591
:101A6000892388B93EC02034310591F42AB18F70A2
:101A70009927D80102C0AA0FBB1F8A95E2F7CD01B2
:101A8000922F982B9AB99BB1809589238BB929C045
:101A90002035310591F42DB18F709927F80102C0DE
:101AA000EE0FFF1F8A95E2F7CF01922F982B9DB979
:101AB0009EB1809589238EB914C02036310589F4F2
:101AC00020B38F709927A80102C0440F551F8A9533
:101AD000E2F7CA01922F982B90BB91B3809589238E
:101AE00081BB50EA5A95F1F7BE016F5F7F4F20E04E
:101AF00030E040E050E0E7E7F2E0DE011196862DAD
:101B000001900D928A95E1F7DB018D919D91BD01C8
:101B1000FC01E07FFF27E032F10511F4E3B113C0CF
:101B2000E033F10511F4E6B10EC0E034F10511F433
:101B3000E9B109C0E035F10511F4ECB104C0E036BB
:101B4000F105B9F4EFB1F0E08F70992702C0F59577
:101B5000E7958A95E2F7E0FD08C0C801042E02C0AF
:101B6000880F991F0A94E2F702C080E090E0282BCA
:101B7000392B4F5F5F4F4C30510509F0BCCFF70157
:101B8000808191818217930721F0318320837092A5
:101B90000B020E94300BF2E0EF0EF11C42EBE41658
:101BA00042E0F40609F026CF80910B028823C9F0A9
:101BB000815080930B02882339F08FE99FE00197D1
:101BC000F1F700C000000DC0E2EBF2E0D5018D910D
:101BD0009D915D0181939193B2EBAB16B2E0BB0690
:101BE000A9F70E94F50781E0A2960FB6F894DEBF30
:101BF0000FBECDBFDF91CF911F910F91FF90EF905E
:101C0000DF90CF90BF90AF909F908F907F906F901C
:101C10005F900895E82FF0E0EE0FFF1FEE54FD4FA8
:101C2000808191810895089580918C0381608093D3
:101C30008C030C94B82880918C038E7F80938C0346
:101C40000C94B8280E948A28811102C00E9466283C
:101C50000E94B42880938C033E9A809171008D7FFE
:101C60008093710082E0809390008AE180939100DC
:101C700081E08093BE0208958091BE02811102C06E
:101C80000E94220E10920E0310920D03809171009B
:101C90008D7F80937100809190008F77809390006A
:101CA0001092D0021092CF021092070310920803F4
:101CB0001092090310920A03109206031092050372
:101CC000E5EEF2E0A5EDB2E01192119211921192BF
:101CD0001D921D9283E0E530F807B1F70895CF9289
:101CE000DF92EF92FF920F931F93CF93DF93209198
:101CF000CF02222309F484C06B017C018091BE02D3
:101D0000811102C00E94220E05E013E0C7E0D0E07E
:101D1000A7019601F80192918291729162918F01CF
:101D20000E94F42D811131C0FE01EE0FFF1FEE0F56
:101D3000FF1FEB51FD4F1082118212821382DE01D0
:101D4000AA0FBB1FAB52BD4F11961C921E92C730FB
:101D5000D105E9F0219644815581668177814083E0
:101D600051836283738314821582168217821296BE
:101D70008D919C91139711969C938E9313961C9220
:101D80001E92129734961296E2CF219708F6809110
:101D90000D0390910E03019797FD05C090930E03DC
:101DA00080930D0304C010920E0310920D038091D6
:101DB0000D0390910E0320910B0330910C03281713
:101DC000390724F010920C0310920B03892BC1F4F5
:101DD000809171008D7F80937100809190008F774A
:101DE0008093900010920703109208031092090349
:101DF00010920A0310920603109205031092CF026C
:101E0000DF91CF911F910F91FF90EF90DF90CF90D6
:101E100008951F920F920FB60F9211244F925F9266
:101E20006F927F928F929F92AF92BF92CF92DF92EA
:101E3000EF92FF922F933F934F935F936F937F9314
:101E40008F939F93AF93BF93CF93DF93EF93FF93C2
:101E50008091CF02882309F49BC1C0910D03D091DA
:101E60000E031C161D060CF093C14090BF0250904B
:101E7000C0026090C1027090C20220E030E0A9016F
:101E8000C301B2010E94432F18160CF065C0C13087
:101E9000D10509F452C080910B0390910C03BE014F
:101EA0000E9423317C0190930C0380930B0380905C
:101EB000D1029090D202A090D302B090D40220E040
:101EC00030E040E85FE3C501B4010E94902D6093CB
:101ED000D1027093D2028093D3029093D402F7017F
:101EE000EE0FFF1FEE0FFF1FEB51FD4FA3019201FD
:101EF00060817181828193810E94F82D20E030E021
:101F000040E05EE30E94472F9B01AC01C501B40194
:101F10000E94432F18168CF4C7010196BE010E943F
:101F2000233190930C0380930B031092D1021092F3
:101F3000D2021092D3021092D402E0910B03F091DE
:101F40000C03EE0FFF1FEE0FFF1FEB51FD4F6081E3
:101F5000718182819381D0C0C0900703D090080323
:101F6000E0900903F0900A0320E030E0A901C701E6
:101F7000B6010E94F42D2197882309F4A2C0FE0126
:101F8000EE0FFF1FEE0FFF1FEB51FD4F8080918082
:101F9000A280B380A5019401C701B6010E94F42D6F
:101FA00087FF31C0A501940160E070E08CED93ECF7
:101FB0000E94F82D20E030E040E451E40E94F82D2A
:101FC00020E030E040E05FE30E94472F9B01AC013E
:101FD00060E070E080E090E40E94AA2F9B01AC01D9
:101FE000C501B4010E94472F9B01AC01C701B60196
:101FF0000E94F42D87FF07C0A701960160E070E002
:102000008CED93E439C0A5019401C701B6010E948B
:10201000432F18160CF055C0A501940160E070E044
:102020008CED93E40E94F82D20E030E040E451E490
:102030000E94F82D20E030E040E05FE30E94472F4F
:102040009B01AC0160E070E080E090E40E94AA2F68
:102050009B01AC01C501B4010E94472F9B01AC015B
:10206000C701B6010E94432F18165CF5A70196011F
:1020700060E070E08CED93EC0E94F82D20E030E001
:1020800040E451E40E94F82D20E030E040E05FE3BE
:102090000E94472F9B01AC0160E070E080E090E47B
:1020A0000E94AA2F9B01AC01C701B6010E94472FD5
:1020B00060930703709308038093090390930A03C6
:1020C00013C0FE01EE0FFF1FEE0FFF1FEB51FD4F80
:1020D00080819181A281B38180930703909308034B
:1020E000A0930903B0930A0360910703709108035A
:1020F0008091090390910A032091BC023091BD02A6
:102100002F3F4FEF340731F02F5F3F4F3093BD0229
:102110002093BC020E9430136B017C0120E034E26A
:1021200044EF51E40E94F42D87FF08C086EFC82ECB
:1021300088E2D82E84EFE82E81E4F82E20E030E00B
:1021400040E051E4C701B6010E94472F9B01AC015A
:1021500060E074E284E79BE40E94F82D6B017C014F
:102160000E94602E709397006093960020910C025D
:1021700030910D0240910E0250910F02C701B6013D
:102180000E94472F0E94602E7093990060939800E0
:102190008091D002882309F433C1C090CB02D09043
:1021A000CC02E090CD02F090CE0220E030E0A90118
:1021B000C701B6010E94432F1816D4F58091BC02C6
:1021C0009091BD028F3F2FEF920729F001969093D7
:1021D000BD028093BC02C701B6010E94301320E00B
:1021E00030E040E051E40E94472F9B01AC0160E0E9
:1021F00074E284E79BE40E94F82D6B017C010E944D
:10220000602E709397006093960020910C0230919D
:102210000D0240910E0250910F02C701B6010E94BB
:10222000472F0E94602E709399006093980008C019
:1022300010929700109296001092990010929800B8
:102240006091C5027091C6026F5F7F4F7093C602A6
:102250006093C502209196003091970080E090E055
:10226000232BF1F0C0919600D09197000E94912EFF
:102270006B017C01BE0180E090E00E94912E9B01E9
:10228000AC016091C7027091C8028091C90290911F
:10229000CA020E94F82D20E03FEF4FE757E410C03C
:1022A0000E94912E6B017C0120E030EE4FEF54E450
:1022B0006091C7027091C8028091C9029091CA02D0
:1022C0000E94472F9B01AC01C701B6010E94432F1A
:1022D00087FD96C08091C3028F5F8093C30290E018
:1022E000209188033091890382179307A0F0809191
:1022F0009303882319F01092C3020DC080917100DE
:102300008D7F80937100809190008F7780939000F3
:102310001092D0027DC08091C402C091C30281118D
:1023200028C0C0908D03D0908E03E0908F03F09072
:10233000900320E030E0A901C701B6010E94432FBD
:102340001816BCF481E08093C4021092CB02109264
:10235000CC021092CD021092CE02C092C702D0924F
:10236000C802E092C902F092CA02C150C093C302EF
:1023700043C01092C4021092BD021092BC02E091C0
:102380008A03F0918B0348E0C49FE00DF11D1124F6
:1023900080819181A281B3818093CB029093CC0202
:1023A000A093CD02B093CE0220E030E040E85EE39F
:1023B00064817581868197810E94472F6B017C0122
:1023C00020E030E048EC52E460911002709111027C
:1023D00080911202909113020E94F82D9B01AC0192
:1023E000C701B6010E94472F6093C7027093C802CD
:1023F0008093C9029093CA021092C6021092C5023D
:1024000080918C0380FD04C01092D0021092CF0204
:10241000FF91EF91DF91CF91BF91AF919F918F91FC
:102420007F916F915F914F913F912F91FF90EF902E
:10243000DF90CF90BF90AF909F908F907F906F90E4
:102440005F904F900F900FBE0F901F901895CF92F6
:10245000DF92EF92FF92CF93DF936B017C01EA0151
:102460008091BE02811102C00E94220E80918C03D5
:1024700080FF46C080910D0390910E0308970CF0E9
:102480003FC0809171008D7F809371008091D00258
:1024900081110E943C0E81E08093CF021092BD0218
:1024A0001092BC0220E030E0A901C701B6010E94F1
:1024B000432F1816DCF480910D0390910E03FC015C
:1024C000EE0FFF1FEE0FFF1FEB51FD4FC082D182B9
:1024D000E282F382FC01EE0FFF1FEB52FD4FD1832E
:1024E000C083019690930E0380930D038091710039
:1024F000826080937100809190008068809390004A
:10250000DF91CF91FF90EF90DF90CF9008958F9261
:102510009F92AF92BF92CF92DF92EF92FF920F9372
:102520001F93CF93DF93EC017B01D42E4801590117
:102530008091BE02811102C00E94220E80918C0304
:1025400080FF6BC0809171008D7F809371008091BE
:10255000CF0281110E943C0E81E08093D002D09383
:102560008B03C0938A03F0928903E0928803D09290
:10257000930380928D0390928E03A0928F03B0926A
:1025800090031092D1021092D2021092D3021092B4
:10259000D4021092C30288819981AA81BB81809361
:1025A000CB029093CC02A093CD02B093CE0220E058
:1025B00030E040E85EE36C817D818E819F810E94E6
:1025C000472F6B017C0120E030E048EC52E4609141
:1025D00010027091110280911202909113020E94D8
:1025E000F82D9B01AC01C701B6010E94472F6093F3
:1025F000C7027093C8028093C9029093CA021092D6
:10260000C6021092C50280917100826080937100B1
:1026100080919000806880939000DF91CF911F910E
:102620000F91FF90EF90DF90CF90BF90AF909F9071
:102630008F90089580910F0390E0019665E070E01F
:102640000E94233180930F03089580910F0390E03F
:10265000019765E070E00E94233180930F03089595
:102660008F929F92AF92BF92CF92DF92EF92FF92A2
:10267000CF93DF936B017C01C091BC02D091BD026E
:10268000BE0180E090E00E94912E4B015C01A70109
:10269000960160E070E08CE594E40E94F82D9B01C7
:1026A000AC01C501B4010E94472F0E94652E4091E4
:1026B0000F03423009F45CC028F4442351F0413048
:1026C000E9F0FBC0433009F481C0443009F4B4C0E0
:1026D000F4C080E090E0A0E0BFE380930C02909310
:1026E0000D02A0930E02B0930F021092BF0210923F
:1026F000C0021092C1021092C202DFC01092BF024B
:102700001092C0021092C1021092C202643171058F
:1027100040F46A307105E0F520E030E040E85EE327
:102720003BC0693C710508F0C0C080E090E00E94A9
:10273000912E20E030E040EA51E40E948F2D20E00D
:1027400030E044E353E40E94F82D9B01AC010E9469
:10275000472F20E030E040E05EE30E94472F9B01DE
:10276000AC0160E070E080E09EE30E948F2D5BC0D2
:102770001092BF021092C0021092C1021092C202C7
:102780006432710578F4FB01EE59FF4F0C94373138
:1027900020E030E040E05FE3C701B6010E94472F30
:1027A0006B017C0180E090E0A0E0BEE380930C022E
:1027B00090930D02A0930E02B0930F027EC0A7016A
:1027C0009601C701B6010E94902DEACF1092BF0278
:1027D0001092C0021092C1021092C2022AE0269FFB
:1027E000A001279F500D1124CA0168EB7BE00E94D5
:1027F0000F31BC016C5D754077FF03C07195619529
:102800007109882777FD8095982F0E94932E2EE3DB
:1028100033EC4EE259E30E94472F20E030E040ECD9
:102820005EE30E94902D60930C0270930D028093E2
:102830000E0290930F0241C01092BF021092C0028C
:102840001092C1021092C202CE0183709927892B87
:10285000E1F0BE016170772780E090E00E94912E48
:1028600020E030E040E05EE30E94472F20E030E0CF
:1028700040E45FE30E94902D60930C0270930D0280
:1028800080930E0290930F020CC080E090E0A0E0D5
:10289000BFE380930C0290930D02A0930E02B093BD
:1028A0000F02C770DD27CD2B41F410920C0210925D
:1028B0000D0210920E0210920F02C701B601DF91B5
:1028C000CF91FF90EF90DF90CF90BF90AF909F900F
:1028D0008F900895809118030895CF93DF9300D0CF
:1028E0001F92CDB7DEB79C0180919803843019F513
:1028F00093E099833B832A839093E9008FEF909133
:10290000E800815095FD06C095ED9A95F1F700001D
:102910008111F5CF8091E80085FF0DC040E050E0C7
:1029200063E070E0CE0101960E94A6168091E80057
:102930008E778093E8000F900F900F90DF91CF91EA
:102940000895CF93DF9300D01F92CDB7DEB72091CB
:102950009803243021F522E029839B838A8383E036
:102960008093E9008FEF9091E800815095FD06C0BB
:1029700095ED9A95F1F700008111F5CF8091E8006F
:1029800085FF0DC040E050E063E070E0CE010196AD
:102990000E94A6168091E8008E778093E8000F9041
:1029A0000F900F90DF91CF910895209198032430DC
:1029B000F1F422E02093E9002FEF3091E80021505C
:1029C00035FD06C035ED3A95F1F700002111F5CF40
:1029D0002091E80025FF0BC040E050E065E070E08A
:1029E0000E94A6168091E8008E778093E8000895F3
:1029F000CF93DF9320919803243039F521E0209381
:102A0000E9002FEF3091E800215035FD06C035ED8B
:102A10003A95F1F700002111F5CF2091E80025FF4C
:102A200014C0EC0140E050E068E070E00E94A6169F
:102A30008091E8008E778093E80088E0FE01A0E1B5
:102A4000B3E001900D928A95E1F7DF91CF9108955F
:102A500080919703811109C00E943B180E94981829
:102A60008091E20084608093E200089510929703C1
:102A70000895089508950C94962742E061EC81E052
:102A80000E94B51742E061EC82E00E94B51742E077
:102A900061EC83E00C94B51780919A03833009F4BC
:102AA00053C030F4813071F0823009F48CC0089545
:102AB0008A3009F478C08B3009F45EC0893009F09F
:102AC0009AC020C080919903813A09F094C0809106
:102AD000E800877F8093E80080919D0390919E039A
:102AE000892B21F468E080E193E003C060E080E09E
:102AF00090E070E00E94F1168091E8008B7780935F
:102B0000E800089580919903813209F074C08091A2
:102B10009D0390919E03892B09F06DC08091E80080
:102B2000877F8093E8008091E80082FD05C0809156
:102B300098038111F8CF5FC08091F1008093180352
:102B40008091E8008B7753C080919903813A09F016
:102B500052C080919D0390919E03892B09F04BC038
:102B60008091E800877F8093E8008091E80080FFF3
:102B7000FCCF80911E0236C0809199038132D9F535
:102B800080919D0390919E03892BA9F58091E80087
:102B9000877F8093E8000E94EA1780919B038093CF
:102BA0001E020C945B2180919903813221F5809162
:102BB000E800877F8093E8000E94EA1780919C03D9
:102BC00080931903089580919903813AA1F480912B
:102BD000E800877F8093E8008091E80080FFFCCFC9
:102BE000809119038093F1008091E8008E778093A3
:102BF000E8000C94EA17089584B7877F84BF88E1C2
:102C00000FB6F89480936000109260000FBE90E0C1
:102C100080E80FB6F89480936100909361000FBE36
:102C20000E948D1B0E943B180E9498188091E20020
:102C300084608093E20078940E941E1B0E948F1B88
:102C400084E192E00E94391B80919803853069F4F9
:102C50000E945027809196038823B1F30E947E271B
:102C6000882391F30E949016EFCF0E94971BECCF20
:102C7000292F332723303105C9F064F42130310581
:102C800081F02230310509F043C084E590E028E16D
:102C90003AE042C021323105F1F02232310541F1F2
:102CA00037C082E190E02CE63AE036C099278130C7
:102CB000910541F08230910541F0892B49F5E4E11D
:102CC000FAE005C0E6EEF9E002C0EAEBF9E0849133
:102CD00090E09F0121C06330D8F4E62FF0E0EE0FC2
:102CE000FF1FE856FD4F2081318189E090E014C03C
:102CF000633070F470E0FB01EE0FFF1FEE56FD4FE6
:102D000020813181FB01E157FD4F808190E004C0BB
:102D100080E090E020E030E0FA01318320830895E4
:102D200080E189BD82E189BD09B400FEFDCF8091BB
:102D3000D8008F7D8093D8008091E00082608093DE
:102D4000E0008091E00081FDFCCF0895CF92DF92FA
:102D5000EF92FF920F931F93CF93DF93EC018B01C0
:102D60006A010E940918811133C0C114D10439F0DD
:102D7000F60180819181081B190BC80FD91FE12C26
:102D8000F12C0115110519F18091E80085FD16C09F
:102D90008091E8008E778093E800C114D10449F057
:102DA000F60180819181E80EF91EF182E08285E0D2
:102DB0000FC00E940918882321F30AC089918093CB
:102DC000F10001501109FFEFEF1AFF0ADACF80E09E
:102DD000DF91CF911F910F91FF90EF90DF90CF90F7
:102DE000089520919F033091A0032617370748F0DC
:102DF0006115710539F42091E8002E772093E800E1
:102E000001C0B90140E061157105A9F12091980355
:102E1000222309F443C0253009F442C02091E80080
:102E200023FD40C02091E80022FD32C02091E8003F
:102E300020FFE9CF4091F3002091F20030E0342BE5
:102E4000FC01CF016115710559F02830310540F4BE
:102E500081918093F100615071092F5F3F4FF1CF55
:102E600041E02830310509F040E02091E8002E775C
:102E70002093E800C8CF4111C9CF0AC080919803C0
:102E8000882361F0853061F08091E80083FD0AC0FD
:102E90008091E80082FFF2CF80E0089582E00895FB
:102EA00083E0089581E0089520919F033091A0036D
:102EB0002617370748F06115710539F42091E800AD
:102EC0002E772093E80001C0B901FC0120E06115D4
:102ED000710591F180919803882309F440C08530F1
:102EE00009F43FC08091E80083FD3DC08091E80077
:102EF00082FD2FC08091E80080FFE9CF2091F30090
:102F00008091F20090E0922B6115710559F08830A4
:102F1000910540F424912093F1003196615071099C
:102F20000196F2CF21E0089709F020E08091E800B7
:102F30008E778093E800CBCF2111CCCF0AC080914F
:102F40009803882361F0853061F08091E80083FD6B
:102F50000AC08091E80082FFF2CF80E0089582E00D
:102F6000089583E0089581E00895982F973058F5EB
:102F70009093E900981739F07091EC002091ED00E2
:102F80005091F00003C0242F762F50E021FF19C08C
:102F90003091EB003E7F3093EB003091ED003D7FB0
:102FA0003093ED003091EB0031603093EB00709383
:102FB000EC002093ED005093F0002091EE0027FFED
:102FC00007C09F5FD3CF8F708093E90081E00895A1
:102FD00080E008958091990387FF11C08091E800F7
:102FE00082FD05C0809198038111F8CF11C08091B6
:102FF000E8008B770BC080919803882349F080917B
:10300000E80080FFF8CF8091E8008E778093E80099
:1030100008952091E4003091E50095E64091EC00A0
:10302000842F817040FF22C08091E80080FD1CC089
:1030300080919803882391F0853091F08091EB0086
:1030400085FD10C04091E4005091E5004217530700
:1030500029F39A01915011F784E0089582E00895D0
:1030600083E0089581E0089580E008954091E800AC
:1030700042FFDECF08950E94A9180E94B118E0EE29
:10308000F0E0808181608083E8EDF0E080818F77DF
:10309000808319BCA7EDB0E08C918E7F8C938081EA
:1030A0008F7E80831092970308950F931F93CF9381
:1030B000DF930E94A9180E94B118C8EDD0E0888162
:1030C0008F77888388818068888388818F7D8883D3
:1030D00019BC1092980310929403109296031092C8
:1030E000950300EE10E0F80180818B7F808388815A
:1030F0008160888342E060E080E00E94B517E1EEE5
:10310000F0E080818E7F8083E2EEF0E0808181605C
:103110008083808188608083F80180818E7F8083B6
:10312000888180618883DF91CF911F910F910895ED
:10313000E8EDF0E080818F7E8083E7EDF0E0808134
:103140008160808384E082BF81E0809397030C9448
:103150005518E8EDF0E080818E7F80831092E200C8
:1031600008951092DA001092E10008951F920F92D4
:103170000FB60F9211242F933F934F935F936F934A
:103180007F938F939F93AF93BF93EF93FF93809120
:10319000E10082FF0BC08091E20082FF07C08091B6
:1031A000E1008B7F8093E1000E941D1B8091DA007B
:1031B00080FF1FC08091D80080FF1BC08091DA0083
:1031C0008E7F8093DA008091D90080FF0DC080E16E
:1031D00089BD82E189BD09B400FEFDCF81E0809305
:1031E00098030E94281505C019BC109298030E94EC
:1031F00036158091E10080FF19C08091E20080FFC8
:1032000015C08091E2008E7F8093E2008091E20001
:1032100080618093E2008091D80080628093D80022
:1032200019BC85E0809398030E943A158091E100D3
:1032300084FF30C08091E20084FF2CC080E189BD12
:1032400082E189BD09B400FEFDCF8091D8008F7D59
:103250008093D8008091E1008F7E8093E10080917F
:10326000E2008F7E8093E2008091E2008160809393
:10327000E20080919403882311F084E007C08091DC
:10328000E30087FD02C081E001C083E080939803E2
:103290000E943B158091E10083FF29C08091E200EC
:1032A00083FF25C08091E100877F8093E10082E069
:1032B00080939803109294038091E1008E7F809315
:1032C000E1008091E2008E7F8093E2008091E20035
:1032D00080618093E20042E060E080E00E94B517E8
:1032E0008091F00088608093F0000E943915FF9172
:1032F000EF91BF91AF919F918F917F916F915F916E
:103300004F913F912F910F900FBE0F901F901895E6
:103310001F920F920FB60F9211242F933F934F934A
:103320005F936F937F938F939F93AF93BF93CF934D
:10333000DF93EF93FF93C091E900CF708091EC0091
:10334000D82FD17080FDD0E81092E9008091F00074
:10335000877F8093F00078940E94CC191092E90046
:103360008091F00088608093F000CD2BCF70C093E7
:10337000E900FF91EF91DF91CF91BF91AF919F91C4
:103380008F917F916F915F914F913F912F910F900E
:103390000FBE0F901F9018951F93CF93DF93CDB75B
:1033A000DEB7AA970FB6F894DEBF0FBECDBFE9E92E
:1033B000F3E088E08E0F9091F10091938E13FBCF94
:1033C0000E944C158091E80083FF1FC180919903F2
:1033D00090919A03492F50E04A30510508F015C1E9
:1033E000FA01EA57FF4F0C943731803881F0823868
:1033F00009F00BC180919D038F708093E90080914B
:10340000EB0085FB882780F91092E90006C08091C7
:10341000950390919603911182609091E800977FB7
:103420009093E8008093F1001092F100C8C0282F1B
:103430002D7F09F0EAC0882319F0823061F0E5C0E1
:1034400080919B03813009F0E0C0933009F080E067
:10345000809396032BC080919B03811127C080919C
:103460009D038F7009F4D1C08093E9002091EB0097
:1034700020FF1CC0933021F48091EB00806214C0C7
:103480009091EB0090619093EB0021E030E0A90176
:1034900002C0440F551F8A95E2F74093EA0010924C
:1034A000EA008091EB0088608093EB001092E900C5
:1034B0008091E800877F86C08111A7C010919B038F
:1034C0001F778091E3008078812B8093E3008091C7
:1034D000E800877F8093E8000E94EA178091E80067
:1034E00080FFFCCF8091E30080688093E30011119E
:1034F00002C082E001C083E08093980386C08058B8
:10350000823008F082C080919B0390919C038C3D97
:1035100053E0950779F583E08A838AE289834FB780
:10352000F894DE01139620E03EE051E2E32FF0E054
:1035300050935700E49120FF03C0E295EF703F5F86
:10354000EF708E2F90E0EA3010F0C79601C0C09661
:103550008D939D932F5F243149F74FBF8091E800F1
:10356000877F8093E8006AE270E0CE0101960E94B6
:10357000F11614C0AE014F5F5F4F60919D030E9432
:103580003816BC01009709F440C09091E800977F7D
:103590009093E80089819A810E9454178091E800F5
:1035A0008B778093E80031C0803879F58091E8000E
:1035B000877F8093E800809194038093F10080914D
:1035C000E8008E778093E8000E94EA171EC0811100
:1035D0001CC090919B039230C0F48091E800877FDB
:1035E0008093E800909394030E94EA1780919403DB
:1035F000811106C08091E30087FD02C081E001C017
:1036000084E0809398030E943D158091E80083FF39
:103610000AC08091E800877F8093E8008091EB00EA
:1036200080628093EB00AA960FB6F894DEBF0FBEBF
:10363000CDBFDF91CF911F9108950895CF938091D1
:1036400098038823A1F0C091E900CF709091EC001D
:10365000892F817090FD80E8C82B1092E90080913D
:10366000E80083FD0E94CC19CF70C093E900CF9190
:10367000089590931F0380931E030895E0911E0305
:10368000F0911F03309721F00190F081E02D099413
:1036900080E00895E0911E03F0911F03309721F020
:1036A0000280F381E02D09940895E0911E03F091CA
:1036B0001F03309721F00480F581E02D09940895CF
:1036C00020911C0330911D038217930771F0909392
:1036D0001D0380931C03E0911E03F0911F0330979C
:1036E00021F00680F781E02D0994089520911A03B6
:1036F00030911B038217930771F090931B03809303
:103700001A03E0911E03F0911F03309721F000840B
:10371000F185E02D0994089508950C948C1B0E9466
:10372000CA270E94F60B0E9450280C94F82C4F9246
:103730005F927F928F929F92AF92BF92CF92DF92D1
:10374000EF92FF920F931F93CF93DF93CDB7DEB726
:103750002A970FB6F894DEBF0FBECDBF0E94D10CE2
:1037600091E2C92E93E0D92E00E010E0AA24A394A0
:10377000B12C702E802F0E940A0E4C01F601419050
:1037800051906F014826592641145104B1F40F5F3E
:103790001F4F0530110569F78FEF89838A831B82DC
:1037A0000E94D3278160782F9D838C8349815A8121
:1037B0006B818D810E94501C3AC08091770381FDFE
:1037C0000E94130E20E030E07501022E02C0EE0CC4
:1037D000FF1C0A94E2F7C70184219521892B09F186
:1037E0002E837F828E209F2091E0892809F490E02B
:1037F00098870E94D3278160782F9A8789874E8186
:103800005F8168858A850E94501C000F111FF80196
:10381000EF5DFC4F80819181E826F926F182E082FC
:1038200006C02F5F3F4F2C30310571F6B0CF0E949C
:10383000372A109120030E943E1B1817D9F00E94CE
:103840003E1B809320032A960FB6F894DEBF0FBE6E
:10385000CDBFDF91CF911F910F91FF90EF90DF903F
:10386000CF90BF90AF909F908F907F905F904F9040
:103870000C942E0B2A960FB6F894DEBF0FBECDBF68
:10388000DF91CF911F910F91FF90EF90DF90CF903C
:10389000BF90AF909F908F907F905F904F900895D2
:1038A000CF93DF93CDB7DEB72B970FB6F894DEBF7B
:1038B0000FBECDBF4F83588769877A878B87DE011C
:1038C000119686E0FD0111928A95E9F785E0FE01E7
:1038D000379601900D928A95E1F749815A816B8163
:1038E0007C818D819E810E94F5232B960FB6F894E2
:1038F000DEBF0FBECDBFDF91CF910895CF93882358
:1039000009F4C2C0C82F823859F40E943E1B81FDC1
:10391000BBC089E30E949E260E94212789E30CC038
:10392000833879F40E943E1B80FDAEC083E50E947F
:103930009E260E94212783E50E94BB26CF910C94EE
:103940002127843859F40E943E1B82FD9DC087E4E4
:103950000E949E260E94212787E4EECF8CEF8C0FD9
:10396000813A48F48C2F0E94602C81118DC08C2FDD
:103970000E949E26E3CF80E28C0F883048F4C77007
:1039800081E001C0880FCA95EAF70E94DA26D6CFF7
:103990008BE58C0F833078F4C53A29F0C63A31F0C4
:1039A00083E890E005C081E890E002C082E890E002
:1039B000CF910C94601B88E58C0F833108F064C0B4
:1039C000C83A39F1C93A41F1CA3A49F1CB3A51F111
:1039D000CC3A59F1CD3A61F1C03B69F1CE3A71F17F
:1039E000CF3A79F1C13B81F1C23B89F1C33B91F1FF
:1039F000C43B99F1C53BA1F1C63BA9F1C73BB1F16D
:103A0000C83BB9F1C93BC1F1CA3BC9F180E090E0C4
:103A100038C082EE90E035C089EE90E032C08AEE88
:103A200090E02FC085EB90E02CC086EB90E029C0A1
:103A300087EB90E026C08CEC90E023C08DEC90E00A
:103A400020C083E891E01DC08AE891E01AC082E9B5
:103A500091E017C084E991E014C081E292E011C0C6
:103A600083E292E00EC084E292E00BC085E292E035
:103A700008C086E292E005C087E292E002C08AE2D6
:103A800092E0CF910C94761BCF910895882309F48E
:103A90004BC0823859F40E943E1B81FF45C089E328
:103AA0000E949E260E94212789E30CC0833871F46E
:103AB0000E943E1B80FF38C083E50E949E260E9424
:103AC000212783E50E94BB260C942127843859F4D2
:103AD0000E943E1B82FF28C087E40E949E260E940F
:103AE000212787E4EFCF9CEF980F913A58F390E2AB
:103AF000980F983050F4877091E001C0990F8A9523
:103B0000EAF7892F0E94E026DFCF9BE5980F9330DC
:103B100020F480E090E00C94601B885A833120F4FC
:103B200080E090E00C94761B0895882321F00E9499
:103B3000DA260C9421270895882321F00E94E0269C
:103B40000C9421270895BF92CF92DF92EF92FF92BB
:103B50000F931F93CF93DF9300D000D000D0CDB749
:103B6000DEB725E0FC01DE01119601900D922A9549
:103B7000E1F7FC01D08011810281258122952F700F
:103B800043815481452B09F472C31F3F21F4FFEF99
:103B9000DF1609F46CC37C012E830E94F707D982DB
:103BA0001A8369817A81802F0E949A26182FB92E54
:103BB0000E944F260E9416252E81002319F00E9494
:103BC000F7262E81EB2DE295EF70F0E0E057FF4FE6
:103BD0000C9437318B2D807F9B2D9F70F92E88237D
:103BE00019F0F29480EFF822002389F0FF2009F405
:103BF0007CC280E2810F883020F48F2D0E94DA266B
:103C000003C08F2D0E94EA260E9421276EC2812FB9
:103C10000E94461DFF2009F42AC3105E8F2D183024
:103C200018F40E94E02602C00E94F02626960FB6E5
:103C3000F894DEBF0FBECDBFDF91CF911F910F91E2
:103C4000FF90EF90DF90CF90BF900C9421278B2DA9
:103C5000807F9B2D9F70803211F4892F03C0892FA4
:103C60008295807F112319F0113011F12BC00023B0
:103C7000A9F0222389F1213079F526960FB6F89420
:103C8000DEBF0FBECDBFDF91CF911F910F91FF908F
:103C9000EF90DF90CF90BF900C940A27222319F069
:103CA000213009F4E4C28E830E940D278E819BC1CE
:103CB000002321F0263008F0DAC20EC0253008F0CB
:103CC000D6C291C10023C9F0222331F0F7019581BA
:103CD00090FF0BC29F70958326960FB6F894DEBFB7
:103CE0000FBECDBFDF91CF911F910F91FF90EF904D
:103CF000DF90CF90BF900C94951D222309F473C1DF
:103D000009C22B2D26952695237030E0211531050B
:103D100021F021303105D1F0AAC2002321F0812FFA
:103D20009B2D937002C080E090E026960FB6F89429
:103D3000DEBF0FBECDBFDF91CF911F910F91FF90DE
:103D4000EF90DF90CF90BF900C94601B002321F088
:103D5000812F9B2D937002C080E090E026960FB6D5
:103D6000F894DEBF0FBECDBFDF91CF911F910F91B1
:103D7000FF90EF90DF90CF90BF900C94761B812F37
:103D8000002319F00E943F2902C00E94A72926960D
:103D90000FB6F894DEBF0FBECDBFDF91CF911F915C
:103DA0000F91FF90EF90DF90CF90BF900C942C2A52
:103DB0008B2D837009F07BC0011159C2812F829530
:103DC00086958770880F880F912F9F70C92ED12CF0
:103DD000E12CF12C082E04C0CC0CDD1CEE1CFF1CC9
:103DE0000A94D2F714FF12C04FE050E060E070E098
:103DF00004C0440F551F661F771F8A95D2F7CB0169
:103E0000BA01609570958095909503C060E070E070
:103E1000CB012B2D269526952370422F50E0423062
:103E20005105D9F04330510569F16C297D298E295E
:103E30009F294130510551F126960FB6F894DEBF07
:103E40000FBECDBFDF91CF911F910F91FF90EF90EB
:103E5000DF90CF90BF900C943D256C297D298E2951
:103E60009F2926960FB6F894DEBF0FBECDBFDF9117
:103E7000CF911F910F91FF90EF90DF90CF90BF9067
:103E80000C9459250E943D25C701B60126960FB610
:103E9000F894DEBF0FBECDBFDF91CF911F910F9180
:103EA000FF90EF90DF90CF90BF900C9421250023DE
:103EB00019F08B2D817001C08695882309F4D7C134
:103EC000812F829586958770880F880F912F9F701C
:103ED000C92ED12CE12CF12C082E04C0CC0CDD1CF9
:103EE000EE1CFF1C0A94D2F714FF12C04FE050E002
:103EF00060E070E004C0440F551F661F771F8A956D
:103F0000D2F7CB01BA01609570958095909503C06A
:103F100060E070E0CB012B2D269526952370422F73
:103F200050E042305105D9F04330510569F16C2918
:103F30007D298E299F294130510551F126960FB6D2
:103F4000F894DEBF0FBECDBFDF91CF911F910F91CF
:103F5000FF90EF90DF90CF90BF900C9417266C29C4
:103F60007D298E299F2926960FB6F894DEBF0FBEB5
:103F7000CDBFDF91CF911F910F91FF90EF90DF9018
:103F8000CF90BF900C9433260E941726C701B6012C
:103F900026960FB6F894DEBF0FBECDBFDF91CF914E
:103FA0001F910F91FF90EF90DF90CF90BF900C94F6
:103FB000FB25103F49F118F4103E48F491C0123F20
:103FC00009F453C0E8F1133F09F464C089C01F70BD
:103FD0008B2D8F71002321F00E949425812F7CCEA0
:103FE0000E94B525812F26960FB6F894DEBF0FBE2E
:103FF000CDBFDF91CF911F910F91FF90EF90DF9098
:10400000CF90BF900C949C1D0023B1F0253008F098
:104010002EC18B2D8F7126960FB6F894DEBF0FBE82
:10402000CDBFDF91CF911F910F91FF90EF90DF9067
:10403000CF90BF900C94DA25263008F018C1E9CF54
:104040000023A9F08B2D8F7126960FB6F894DEBF52
:104050000FBECDBFDF91CF911F910F91FF90EF90D9
:10406000DF90CF90BF900C949425002359F38B2DB3
:104070008F7126960FB6F894DEBF0FBECDBFDF91CD
:10408000CF911F910F91FF90EF90DF90CF90BF9055
:104090000C94B525002399F08B2D8F7126960FB6C1
:1040A000F894DEBF0FBECDBFDF91CF911F910F916E
:1040B000FF90EF90DF90CF90BF900C947F252696D5
:1040C0000FB6F894DEBF0FBECDBFDF91CF911F9129
:1040D0000F91FF90EF90DF90CF90BF900C947525DB
:1040E0000023A9F0222309F4ADCF812F26960FB625
:1040F000F894DEBF0FBECDBFDF91CF911F910F911E
:10410000FF90EF90DF90CF90BF900C947E1C222305
:1041100009F4ADCF812F26960FB6F894DEBF0FBEFF
:10412000CDBFDF91CF911F910F91FF90EF90DF9066
:10413000CF90BF900C94461D4B2D4F70612FC7013F
:104140000E942F0626960FB6F894DEBF0FBECDBF95
:10415000DF91CF911F910F91FF90EF90DF90CF9063
:10416000BF900C949924011182C09B2D9F70492F00
:1041700050E04230510509F443C0C4F441155105E3
:1041800071F14130510509F072C026960FB6F894CE
:10419000DEBF0FBECDBFDF91CF911F910F91FF907A
:1041A000EF90DF90CF90BF900C94202D43305105BD
:1041B000C1F14430510509F05AC0812F26960FB63F
:1041C000F894DEBF0FBECDBFDF91CF911F910F914D
:1041D000FF90EF90DF90CF90BF900C94722D2696B9
:1041E0000FB6F894DEBF0FBECDBFDF91CF911F9108
:1041F0000F91FF90EF90DF90CF90BF900C94092D1E
:1042000026960FB6F894DEBF0FBECDBFDF91CF91DB
:104210001F910F91FF90EF90DF90CF90BF900C9483
:104220003C2D26960FB6F894DEBF0FBECDBFDF91B2
:10423000CF911F910F91FF90EF90DF90CF90BF90A3
:104240000C944F2D4B2D4F70612FC70126960FB642
:10425000F894DEBF0FBECDBFDF91CF911F910F91BC
:10426000FF90EF90DF90CF90BF900C94F9072696C7
:104270000FB6F894DEBF0FBECDBFDF91CF911F9177
:104280000F91FF90EF90DF90CF90BF9008950E9424
:10429000F7260E9407270E94CC260E9421270E9411
:1042A000DD2A0E942C2A80E090E00E94601B80E0C2
:1042B00090E00C94761B0E94E7260C9447210E9404
:1042C0008F26292F22952F7030E02C3031054CF4A9
:1042D0002A3031056CF4225031092230310588F43E
:1042E00007C02C30310549F02F30310531F009C0BD
:1042F000803E48F0803F29F406C093FB882780F970
:10430000089580E0089581E00895CF93DF9300D071
:1043100000D01F92CDB7DEB70F900F900F900F9087
:104320000F90DF91CF910895CF93DF9300D000D00D
:1043300000D0CDB7DEB726960FB6F894DEBF0FBE1D
:10434000CDBFDF91CF9108951F93CF93DF93C0919D
:104350002B0316E080912C03C81799F0D0E01C9F26
:10436000F0011D9FF00D1124E35DFC4F4081518150
:1043700062817381848195810E9494212196C77006
:10438000E9CFDF91CF911F91089540915D03509146
:104390005E0360915F03709160038091610390916F
:1043A00062030C9494218091620382958F7009F0CE
:1043B00054C080915F03882309F44FC080912B0380
:1043C000A0912C0360915D0370915E0340916003A6
:1043D00050916103B6E08A1709F43FC090E041159F
:1043E0005105C1F17F3F11F46F3FA1F1B89FF0017A
:1043F000B99FF00D1124E35DFC4F218172132AC097
:104400002081621327C02281211124C0238134819D
:104410002417350710F421503109241B350B283C93
:104420003105C0F4209162032F7020612093620354
:1044300026E0289FF001299FF00D1124EE5CFC4F2F
:1044400080818F70806180838DE593E00E94A31D41
:104450000C94A42101968770BECF0895CF92DF926D
:10446000EF92FF920F931F93CF93DF93CDB7DEB7F9
:1044700062970FB6F894DEBF0FBECDBF8C0185E00A
:10448000F801DE011D9601900D928A95E1F7D801A1
:104490004C9111965C91119712966C91129713960C
:1044A000CD90DC90149730915D0370915E03809104
:1044B000600390916103009709F46BC17F3F19F489
:1044C0003F3F09F466C1E0905F03EE2009F4C0C0ED
:1044D00020916203C816D90628F0F601E81BF90BF3
:1044E000CF0104C0809590958C0D9D1DFF24F39401
:1044F000883C910578F0F12C207F09F0C6C07C2D16
:10450000D98AC88A89890E9485218DE593E00E9415
:10451000A31DB1C0822F807F09F046C0751314C05F
:10452000341312C0611110C02F70206120936203F8
:104530000E94C5218DE593E00E94A31D8091620336
:10454000D80115968C932EC0CD2819F15F3F11F438
:104550004F3FF9F0F62E61111CC080912B03209182
:104560002C0336E0821709F45AC090E0389FF0011E
:10457000399FF00D1124E35DFC4F7181571306C084
:104580007081471303C07281711103C00196877057
:10459000E9CFF62E662309F418C180916203816089
:1045A00080936203F12C11C1751308C0341306C047
:1045B000611104C080916203D801C3C04D875E873A
:1045C0008D859E856A8B0E945F216A898823E1F12F
:1045D0006623D1F120916203822F82958F7090E043
:1045E000029774F080915D0390915E0398878F83AA
:1045F0001986DB86CA862C87CE0107960E94A31DEA
:1046000086E0F801ADE5B3E001900D928A95E1F7FF
:104610000E94D3210E94C521FF24F394D6C04D8768
:104620005E878D859E850E948F26292F22952F706B
:1046300030E0223031050CF0BCC09F7009F0B6C0EC
:10464000805E883008F4C1C0C8010E94A31DE4CF79
:10465000C816D90608F453C0F601E81BF90BCF01C0
:10466000883C910508F450C0F12C7C2DD98AC88A69
:1046700089890E948521EDE5F3E086E0DF011D9246
:104680008A95E9F70E94C521A0C0751314C03413A0
:1046900012C0611110C080916203F8018583C801C6
:1046A0000E94A31D86E0EDE5F3E0DF011D928A95EF
:1046B000E9F7FE2C8AC04D875E878D859E856A8BC3
:1046C0000E945F216A89882309F4BECF662309F41A
:1046D000BBCF20916203822F82958F7090E002976A
:1046E0000CF48ECF80915D0390915E039A83898351
:1046F0001B82DD82CC822E83CE0101967FCF8095F6
:1047000090958C0D9D1DACCFF62E662309F49CCFA1
:1047100075132EC034132CC02091620320FD1FC0DE
:10472000822F82958F70D9F0D80115962C9315970A
:104730008F3049F08F5F982F9295907F822F8F70E6
:10474000892B15968C93C8010E94A31D86E0F80161
:10475000ADE5B3E001900D928A95E1F793CF86E045
:10476000F801ADE5B3E001900D928A95E1F72DC017
:104770004D875E878D859E850E945F21811140CF88
:1047800080916203816080936203C8010E94A31D2F
:104790001CC0662309F458CF4D875E878D859E85A2
:1047A0000E945F21882309F44FCF2ACF811148CF7F
:1047B0000CC0243031050CF047CF9F7009F440CF76
:1047C000F8019581907F09F03BCF8F2D62960FB64F
:1047D000F894DEBF0FBECDBFDF91CF911F910F9137
:1047E000FF90EF90DF90CF9008951F93CF93DF93CA
:1047F000CDB7DEB72C970FB6F894DEBF0FBECDBF96
:104800004F83588769877A878B879C87CE01079665
:104810000E942E22882369F08F8198852A853B8506
:10482000232BF1F19F3F09F063C08F3F09F060C077
:1048300037C086E0FE013796DE01119601900D9299
:104840008A95E1F76F817885EA85FB85309741F19C
:104850007F3F11F46F3F21F120912C0330E0C9011B
:1048600001968770992740912B0350E08417950794
:1048700009F447C069837A83FD83EC8396E0929FB5
:10488000D001939FB00D1124A35DBC4FFE01319662
:1048900001900D929A95E1F780932C030E94A42138
:1048A00016E080912B0390912C038917C1F1189F7A
:1048B000C0011124835D9C4F0E942E22882379F130
:1048C000E0912B031E9FF0011124E35DFC4F40811A
:1048D000518162817381848195810E9494218091AC
:1048E0002B0390E001968770992780932B03D9CFF3
:1048F0004F81588569857A858B859C850E94942196
:10490000CFCF0E945B2110922C0310922B03EDE578
:10491000F3E086E0DF011D928A95E9F7C1CF2C967E
:104920000FB6F894DEBF0FBECDBFDF91CF911F91C0
:104930000895EF92FF920F931F93CF93DF938C0113
:10494000009709F46CC0F12CEE24E394E801219661
:10495000F8018491843740F4843008F051C08130EC
:1049600081F0823019F15BC0853709F444C0A8F1A9
:104970009CE7980F903708F052C08F770E94461D31
:1049800041C00E5F1F4FFE01C49180E28C0F883042
:1049900048F4C7708E2D01C0880FCA95EAF70E94AF
:1049A000FA2614C08C2F0E947E1C2DC00E5F1F4F54
:1049B000FE01C49180E28C0F883058F4C7708E2DB0
:1049C00001C0880FCA95EAF70E9400270E9421279C
:1049D0001AC08C2F0E94461D16C00E5F1F4FFE018D
:1049E000C491CC2381F08FE99FE00197F1F700C0DB
:1049F0000000C150F6CF0E5F1F4FFE01F49003C0C0
:104A00000E947E1C8E018F2D882309F49FCFEFE931
:104A1000FFE03197F1F700C000008150F5CFDF9142
:104A2000CF911F910F91FF90EF900895089560939B
:104A30006703709368038093690390936A030C94EF
:104A400047210F931F9300916703109168032091F2
:104A5000690330916A03DC01CB01802B912BA22BDF
:104A6000B32B8093670390936803A0936903B0937B
:104A70006A031F910F910C9447210F931F9300918C
:104A80006703109168032091690330916A03DC0188
:104A9000CB0180239123A223B323809367039093B8
:104AA0006803A0936903B0936A031F910F910C945C
:104AB00047210F931F930091670310916803209182
:104AC000690330916A03DC01CB0180279127A2277B
:104AD000B3278093670390936803A0936903B0930F
:104AE0006A031F910F910C94472110926303109257
:104AF000640310926503109266030C94472141E011
:104B000050E060E070E004C0440F551F661F771F3F
:104B10008A95D2F7409363035093640360936503CF
:104B2000709366030C94472141E050E060E070E030
:104B300004C0440F551F661F771F8A95D2F78091D6
:104B4000630390916403A0916503B0916603482BC1
:104B5000592B6A2B7B2B4093630350936403609320
:104B60006503709366030C94472141E050E060E0D8
:104B700070E004C0440F551F661F771F8A95D2F757
:104B80004095509560957095809163039091640372
:104B9000A0916503B0916603482359236A237B23C0
:104BA00040936303509364036093650370936603BB
:104BB0000C94472141E050E060E070E004C0440FF5
:104BC000551F661F771F8A95D2F7809163039091D6
:104BD0006403A0916503B0916603482759276A27AB
:104BE0007B27409363035093640360936503709342
:104BF00066030C9447210F931F9300916303109158
:104C000064032091650330916603DC01CB01802BA6
:104C1000912BA22BB32B8093630390936403A093F7
:104C20006503B09366031F910F910C9447210F9376
:104C30001F930091630310916403209165033091E9
:104C40006603DC01CB0180239123A223B32380934D
:104C5000630390936403A0936503B09366031F916D
:104C60000F910C9447210F931F93009163031091B0
:104C700064032091650330916603DC01CB0180273A
:104C80009127A227B3278093630390936403A09393
:104C90006503B09366031F910F910C94472108950B
:104CA000CF92DF92EF92FF920F931F93CF93DF93F8
:104CB0008C01C0906703D0906803E0906903F09086
:104CC0006A038091630390916403A0916503B0919E
:104CD0006603C82AD92AEA2AFB2ACFE1D0E0D70105
:104CE000C6010C2E04C0B695A795979587950A9492
:104CF000D2F780FF06C0B8018C2F0E94530A01979B
:104D000021F4219760F780E001C08C2FDF91CF91D3
:104D10001F910F91FF90EF90DF90CF900895CF9368
:104D2000DF93EC010E945026BE010E94530ADF91DE
:104D3000CF910895CB010E948F26089520911F02E4
:104D400030912002F90132969FEF40E051915817BF
:104D500089F09F3F19F4511101C0942F4F5F4630E5
:104D6000A9F79F3F39F0F901E90FF11D97FDFA9579
:104D700082830895089520911F0230912002F90145
:104D80003296285F3F4F9081981301C01082319670
:104D9000E217F307C1F7089581E090E0E0911F0268
:104DA000F0912002E80FF91F1082019688309105DA
:104DB000A9F7089590917603892B8093760308953F
:104DC00080959091760389238093760308951092BD
:104DD0007603089590917503892B80937503089548
:104DE000809590917503892380937503089510929F
:104DF0007503089590917403892B8093740308952B
:104E00008095909174038923809374030895109280
:104E10007403089580936B03089510926B030895B3
:104E200080911F0290912002FC0131969C01285F25
:104E30003F4F80E0919191118F5FE217F307D1F717
:104E40000895E0911F02F091200280917603808303
:104E5000E0911F02F0912002908180917503892BCF
:104E60008083E0911F02F091200290818091740371
:104E7000892B808380916B03882361F0E0911F026E
:104E8000F09120029081892B80830E94102781114C
:104E900010926B0380911F02909120020C944A1B88
:104EA00080919803843039F11092780320E488E1EE
:104EB00090E00FB6F894A895809360000FBE209301
:104EC000600080E00E94F60580E00E942E0B83B710
:104ED000817F846083BF83B7816083BF7894889526
:104EE00083B78E7F83BF88E10FB6F894809360000C
:104EF000109260000FBE089508950895CF9380E04A
:104F00000E94F6050E947C270E94D10C0E947D27FA
:104F1000C0E08C2F0E940A0E892B29F4CF5FC53088
:104F2000C1F780E001C081E0CF9108950E945B212C
:104F300080E00E94F6050E94F82C0E943E1B0C9413
:104F40002E0B1F920F920FB60F9211248F939F93E7
:104F5000AF93BF9380917803811113C0809179033F
:104F600090917A03A0917B03B0917C034196A11D9F
:104F7000B11D8093790390937A03A0937B03B09340
:104F80007C03BF91AF919F918F910F900FBE0F90B7
:104F90001F90189582E084BD93E095BD9AEF97BD70
:104FA00080936E0008952FB7F894809179039091C3
:104FB0007A03A0917B03B0917C032FBF0895CF9219
:104FC000DF92EF92FF920F931F932FB7F8944091C7
:104FD000790350917A0360917B0370917C032FBF1A
:104FE0006A017B01EE24FF248C0120E030E0C01632
:104FF000D106E206F30610F4415051099A01281B2C
:10500000390BC9011F910F91FF90EF90DF90CF9066
:1050100008951F920F920FB60F9211248F939F93B2
:10502000AF93BF938091790390917A03A0917B0312
:10503000B0917C030196A11DB11D809379039093DB
:105040007A03A0937B03B0937C03BF91AF919F91B0
:105050008F910F900FBE0F901F9018950E943B18D4
:10506000F8942FEF87EA91E6215080409040E1F7D5
:1050700000C0000087E090EBDC018093A3039093D5
:10508000A403A093A503B093A6039CE088E10FB608
:10509000F894A895809360000FBE90936000FFCFB6
:1050A0000E948A28811102C00E9466280E949528C9
:1050B000809377030E94A2288093A1030E949928DD
:1050C000682F70E080E090E00C9417256DEE7EEF85
:1050D00080E090E00E945D3160E082E090E00E941C
:1050E0004B3160E083E090E00E944B3160E084E06F
:1050F00090E00E944B3160E085E090E00E944B31EF
:1051000060E086E090E00E944B316FEF87E090E036
:105110000C944B3180E090E00E94453121E08D3EBF
:105120009E4F09F020E0822F089582E090E00C94D9
:105130003D3183E090E00C943D31682F83E090E0B6
:105140000C944B3184E090E00C943D31682F84E066
:1051500090E00C944B3186E090E00C943D31682F48
:1051600086E090E00C944B3187E090E00C943D3168
:10517000682F87E090E00C944B3180917F0380FF93
:105180000BC06091240285E0689FB00111247595E1
:105190006795759567952BC081FF09C060912402C2
:1051A00085E0689FB00111247595679520C082FF46
:1051B00007C06091240285E0689FB001112417C0E8
:1051C000909180039923D1F060912302961788F77C
:1051D0002091240285E0289F90011124929FA00134
:1051E000939F500D112470E0CA010E942331603852
:1051F000710540F46115710539F002C065E070E099
:10520000862F08958FE7089581E0089580917F03A8
:1052100080FF08C06091220270E0759567957595D2
:10522000679521C081FF06C06091220270E07595EC
:10523000679519C082FF04C06091220270E010C01F
:10524000909180039923C1F0609121029617A0F7F5
:1052500080912202899FC001112470E00E942331B5
:105260006038710528F46115710521F0862F0895C5
:105270008FE7089581E0089561E070E0F4CF803F0A
:1052800021F40E94BD28819504C0813F29F40E9429
:10529000BD28809383030895823F21F40E94BD2896
:1052A000819504C0833F29F40E94BD288093820326
:1052B0000895893F19F40E94062905C08A3F31F4F8
:1052C0000E94062981958093840308958B3F21F4E1
:1052D0000E940629819504C08C3F29F40E9406296A
:1052E000809385030895843F21F480918103816038
:1052F00017C0853F21F480918103826011C0863FF1
:1053000021F48091810384600BC0873F21F4809158
:105310008103886005C0883F31F4809181038061FA
:105320008093810308958D3F21F480917F038160F4
:105330000BC08E3F21F480917F03826005C08F3FB8
:1053400029F480917F03846080937F030895803FD8
:1053500039F48091830387FF6CC01092830369C086
:10536000813F29F4809183031816BCF362C09091A9
:105370008203823F29F497FF5CC01092820359C0D8
:10538000833F19F41916CCF354C0893F41F480913E
:10539000840318160CF04DC0109284034AC08A3F53
:1053A00029F48091840387FF44C0F6CF8B3F39F402
:1053B0008091850387FF3DC0109285033AC08C3FE2
:1053C00029F4809185031816BCF333C0843F21F47F
:1053D000809181038E7F17C0853F21F480918103E6
:1053E0008D7F11C0863F21F4809181038B7F0BC09C
:1053F000873F21F480918103877F05C0883F31F486
:10540000809181038F7E8093810313C08D3F21F4AF
:1054100080917F038E7F0BC08E3F21F480917F03AC
:105420008D7F05C08F3F29F480917F038B7F809310
:105430007F038091820381110EC0809183038111CB
:105440000AC080918403811106C080918503811177
:1054500002C010928003089581E893E00E94551BDA
:105460000E94D32790937E0380937D0308951F931A
:10547000CF93DF9380917D0390917E030E94DF277D
:10548000AC0190918003992321F02091250230E016
:1054900006C0209126028AE0289F9001112442171D
:1054A000530708F486C080918203C0918303D09192
:1054B000840310918503811107C0C11176C0D111F9
:1054C00074C0111172C075C09F3F19F09F5F909317
:1054D0008003181624F40E94BD28809382038091D3
:1054E000820387FF05C00E94BD28819580938203B7
:1054F0001C1624F40E94BD288093830380918303AB
:1055000087FF05C00E94BD28819580938303609129
:105510008203662339F1C0918303CC2319F17727E5
:1055200067FD7095872F972F0E94932E23E333E317
:1055300043E35FE30E94472F0E94602E6093820343
:105540006C2F772767FD7095872F972F0E94932EDA
:1055500023E333E343E35FE30E94472F0E94602E7F
:10556000609383031D1624F40E940629809384030C
:105570008091840387FF05C00E940629819580934E
:105580008403111624F40E940629809385038091D8
:10559000850387FF05C00E940629819580938503B6
:1055A000DF91CF911F910C942C2A9F3F09F08ECF51
:1055B00096CFDF91CF911F910895E1E8F3E085E068
:1055C000DF011D928A95E9F71092800310927F0304
:1055D0000895833081F128F4813059F08230D1F080
:1055E0000895853009F449C0B8F1863009F456C0F1
:1055F000089580912602262F30E0280F311D2F3F7D
:10560000310524F4680F6093260208958FEF80938C
:105610002602089580912502262F30E0280F311DA3
:105620002F3F310524F4680F6093250208958FEF12
:1056300080932502089580912402262F30E0280FC0
:10564000311D2F3F310524F4680F60932402089523
:105650008FEF80932402089580912302262F30E05B
:10566000280F311D2F3F310524F4680F609323026A
:1056700008958FEF80932302089580912202262FB0
:1056800030E0280F311D2F3F310524F4680F60935F
:10569000220208958FEF80932202089580912102C3
:1056A000262F30E0280F311D2F3F310524F4680FDD
:1056B0006093210208958FEF809321020895833033
:1056C00011F128F4813049F0823091F0089585304D
:1056D00081F120F18630C1F108958091260268178A
:1056E00020F4861B809326020895109226020895C6
:1056F00080912502681720F4861B80932502089567
:1057000010922502089580912402681720F4861BC8
:105710008093240208951092240208958091230218
:10572000681720F4861B80932302089510922302A9
:10573000089580912202681720F4861B809322022C
:10574000089510922202089580912102681720F492
:10575000861B8093210208951092210208950F93D1
:105760001F938732D8F58E3108F087C08E3009F448
:1057700071C098F4873009F45BC08B3009F491C094
:10578000863009F095C080917703817F8E7F80936A
:10579000770381E0809387038CC0863109F481C050
:1057A00068F4803109F084C08091770383FB22275D
:1057B00020F991E0922790FB83F955C0893109F4D3
:1057C00070C08B3109F074C08091770381FB222770
:1057D00020F991E0922790FB81F945C0883309F4C4
:1057E00060C050F4893209F45EC0853309F45BC0AF
:1057F000873209F458C05CC0833409F454C028F4DB
:105800008A3308F455C0895339C0883409F050C030
:105810000E945B210E94D6070FEF13ED20E3015099
:1058200010402040E1F700C000000E942E2839C03F
:1058300090917703892F8095817080FB90F929F0F2
:10584000966098609093770334C0997F977F909388
:10585000770327C08091770382FB222720F991E00C
:10586000922790FB82F9809377039923D1F080915E
:10587000770381608093770314C08D5141E050E03D
:1058800060E070E08A019B0104C0000F111F221F1D
:10589000331F8A95D2F7C901B8010E9417250E94CB
:1058A0005B2181E006C061E070E080E090E0F5CF30
:1058B00080E01F910F91089580E0089580E00895A1
:1058C000CF93C82F80918703813069F018F0823020
:1058D000C9F184C0E0911F02F091200280818232E0
:1058E00009F07EC007C0E0911F02F0912002808184
:1058F000823261F48C2F0E945C2C811104C08C2FA9
:105900000E94AF2B1DC081E090E01AC08C2F0E9436
:105910005E2C811114C0C43179F048F4CB3079F099
:10592000C03109F061C082E08093870308C0C932AA
:1059300019F0C83321F058C01092870355C081E098
:10594000817054C0C93291F120F5C43179F1B0F4BD
:10595000C73009F047C08EE18093260282E380932E
:1059600025028AE08093240284E18093230288E068
:105970008093220288E28093210234C0CE51C63047
:1059800088F5EC2FF0E0E256FD4F8081809386038E
:1059900029C0CE34E9F020F4CB3421F56AE013C0FD
:1059A000C13579F0C235F1F461E00DC08091860314
:1059B000882319F01092860315C081E08093870335
:1059C00015C061E006C0809186030E94E92A0AC0E2
:1059D0006AE0809186030E945F2B04C010928703C7
:1059E00080E004C081E002C080E0AACFCF9108959A
:1059F0000E948A28811102C00E9466280E94AB285A
:105A00008093A20380FF02C0869501C080E00C94C1
:105A1000F6058091A203982F9695292F30E0233028
:105A200031054CF49F5F990F8170892B81608093C1
:105A3000A2030E94AF288091A20386950C94F605DC
:105A40008091A203982F969591F09158990F8170AB
:105A5000892B8093A2038E7F91E009F490E08091DE
:105A6000A20390FB80F98093A2030E94AF2880914B
:105A7000A20386950C94F6058091A203982F909529
:105A800090FB80F98093A2030E94AF288091A2032B
:105A900080FF02C0869501C080E00C94F6059091CD
:105AA000A203892F86958F5F8F779170843028F4B9
:105AB000880F892B8093A20302C09093A203809148
:105AC000A2038E7F91E009F490E08091A20390FB05
:105AD00080F98093A2030E94AF288091A20386954B
:105AE0000C94F6052091A203922F96958927982F62
:105AF000990F822F8170892B8093A2038E7F91E072
:105B000009F490E08091A20390FB80F98093A203B6
:105B10000E94AF288091A20386950C94F6055058F8
:105B2000BB27AA270ED075C166D130F06BD120F00B
:105B300031F49F3F11F41EF45BC10EF4E095E7FBD6
:105B400051C1E92F77D180F3BA1762077307840731
:105B5000950718F071F49EF58FC10EF4E0950B2EA9
:105B6000BA2FA02D0B01B90190010C01CA01A001AF
:105B70001124FF27591B99F0593F50F4503E68F10A
:105B80001A16F040A22F232F342F4427585FF3CF4B
:105B9000469537952795A795F0405395C9F77EF41C
:105BA0001F16BA0B620B730B840BBAF09150A1F065
:105BB000FF0FBB1F661F771F881FC2F70EC0BA0FEB
:105BC000621F731F841F48F4879577956795B79573
:105BD000F7959E3F08F0B3CF9395880F08F099276B
:105BE000EE0F979587950895D9D008F481E0089530
:105BF0000CD00FC107D140F0FED030F021F45F3F50
:105C000019F0F0C0511139C1F3C014D198F39923A0
:105C1000C9F35523B1F3951B550BBB27AA27621770
:105C20007307840738F09F5F5F4F220F331F441FB5
:105C3000AA1FA9F333D00E2E3AF0E0E830D09150ED
:105C40005040E695001CCAF729D0FE2F27D0660FDA
:105C5000771F881FBB1F261737074807AB07B0E819
:105C600009F0BB0B802DBF01FF2793585F4F2AF02F
:105C70009E3F510568F0B6C000C15F3FECF3983E0F
:105C8000DCF3869577956795B795F7959F5FC9F78C
:105C9000880F911D9695879597F90895E1E0660F15
:105CA000771F881FBB1F621773078407BA0720F08E
:105CB000621B730B840BBA0BEE1F88F7E0950895F7
:105CC00004D06894B111D9C00895BCD088F09F5712
:105CD00090F0B92F9927B751A0F0D1F0660F771F38
:105CE000881F991F1AF0BA95C9F712C0B13081F018
:105CF000C3D0B1E00895C0C0672F782F8827B85F60
:105D000039F0B93FCCF3869577956795B395D9F778
:105D10003EF490958095709561957F4F8F4F9F4F82
:105D20000895E89409C097FB3EF49095809570958E
:105D300061957F4F8F4F9F4F9923A9F0F92F96E9D7
:105D4000BB279395F695879577956795B795F1114C
:105D5000F8CFFAF4BB0F11F460FF1BC06F5F7F4FE9
:105D60008F4F9F4F16C0882311F096E911C07723FB
:105D700021F09EE8872F762F05C0662371F096E804
:105D8000862F70E060E02AF09A95660F771F881FD3
:105D9000DAF7880F9695879597F90895990F000877
:105DA000550FAA0BE0E8FEEF16161706E807F907ED
:105DB000C0F012161306E407F50798F0621B730B88
:105DC000840B950B39F40A2661F0232B242B252B09
:105DD00021F408950A2609F4A140A6958FEF811DAC
:105DE000811D089597F99F6780E870E060E008954D
:105DF0009FEF80EC089500240A94161617061806E3
:105E00000906089500240A941216130614060506BE
:105E10000895092E0394000C11F4882352F0BB0F4F
:105E200040F4BF2B11F460FF04C06F5F7F4F8F4FB2
:105E30009F4F089557FD9058440F551F59F05F3FED
:105E400071F04795880F97FB991F61F09F3F79F09C
:105E500087950895121613061406551FF2CF46951E
:105E6000F1DF08C0161617061806991FF1CF8695A0
:105E70007105610508940895E894BB276627772784
:105E8000CB0197F908958ADF08F48FEF08950BD0BE
:105E9000C0CFB1DF28F0B6DF18F0952309F0A2CF0C
:105EA000A7CF1124EACFC6DFA0F3959FD1F3950FBA
:105EB00050E0551F629FF001729FBB27F00DB11D8E
:105EC000639FAA27F00DB11DAA1F649F6627B00D1E
:105ED000A11D661F829F2227B00DA11D621F739F07
:105EE000B00DA11D621F839FA00D611D221F749F15
:105EF0003327A00D611D231F849F600D211D822F5C
:105F0000762F6A2F11249F5750408AF0E1F08823A2
:105F10004AF0EE0FFF1FBB1F661F771F881F9150AF
:105F20005040A9F79E3F510570F05CCFA6CF5F3F70
:105F3000ECF3983EDCF3869577956795B795F795E2
:105F4000E7959F5FC1F7FE2B880F911D969587956A
:105F500097F90895FA01EE0FFF1F309621053105DC
:105F600099F16115710561F48038BFE39B0749F130
:105F700068949038810561F08038BFEF9B0741F04D
:105F8000992342F5FF3FE1053105210511F1E89420
:105F90000894E795D901AA2329F4AB2FBE2FF85F07
:105FA000D0F310C0FF5F70F4A695E0F7F73950F01A
:105FB00019F0FF3A38F49F779F930CD00F9007FCAD
:105FC000905808953EF014CF60E070E080E89FE3C1
:105FD00008954FE79F775F934F933F932F939ED002
:105FE0002F913F914F915F9152DF05C019F40EF050
:105FF000F9CE42CFFDCE26DFC8F39638C0F707F8BA
:106000000F92E8942BE33AEA48EB5FE74EDF0F92FA
:106010000F920F924DB75EB70F92C0D0E0E4F1E05F
:1060200016D04F915F91EF91FF91E595EE1FFF1F05
:1060300049F0FE57E0684427EE0F441FFA95E1F758
:106040004195550B32D00F9007FE26C00895DF937F
:10605000CF931F930F93FF92EF92DF927B018C01FE
:10606000689405C0DA2EEF011EDFFE01E894A591C9
:106070002591359145915591AEF3EF0162DDFE0119
:106080009701A801DA9479F7DF90EF90FF900F91D4
:106090001F91CF91DF9108959B01AC0160E070E00A
:1060A00080E89FE3A5CD9ECEACC0CCDEE8F399237B
:1060B000D9F3940F511DBBF39150504094F059F017
:1060C000882332F0660F771F881F91505040C1F728
:1060D0009E3F510544F7880F911D9695879597F936
:1060E00008955F3FACF0983E9CF0BB27869577956E
:1060F0006795B79508F4B1609395C1F7BB0F58F752
:1061000011F460FFE8CF6F5F7F4F8F4F9F4FE3CF5A
:10611000B4CE0EF076C06CCE689464CE93DEC8F335
:106120009923D1F3C6F3DF93CF931F930F93FF927D
:10613000C92FDD2788232AF02197660F771F881F34
:10614000DAF720E030E040E85FEB9FE3883920F0A9
:10615000803E30F021968F77E3DCE8E6F1E003C083
:10616000DFDCE5E9F1E073DF8B01BE01EC01FB2E22
:106170006F5771097595771F880B990BD4DD28E14E
:1061800032E741E35FE38FDEAF2D9801AE01FF9070
:106190000F911F91CF91DF91D4DC3BCEFA01DC014E
:1061A000AA0FBB1F9B01AC01BF5728F4222733273E
:1061B000442750781FC0B75188F4AB2F0024469570
:1061C00037952795011CA395D2F3002069F0220F83
:1061D000331F441FB395DAF30DD0A1CC61307105A4
:1061E000A0E88A07B94630F49B01AC0166277727FF
:1061F00088279078309621F020833183428353831F
:1062000008959F3F31F0915020F4879577956795D9
:10621000B795880F911D9695879597F90895AA1BB4
:10622000BB1B51E107C0AA1FBB1FA617B70710F081
:10623000A61BB70B881F991F5A95A9F780959095B3
:10624000BC01CD01089597FB072E16F4009407D0EA
:1062500077FD09D00E940F3107FC05D03EF49095E0
:1062600081959F4F0895709561957F4F0895EE0F2A
:10627000FF1F0590F491E02D0994F999FECF92BD8E
:1062800081BDF89A992780B50895A8E1B0E042E071
:1062900050E00C946531262FF999FECF92BD81BD57
:1062A000F89A019700B4021639F01FBA20BD0FB654
:1062B000F894FA9AF99A0FBE08950196272F0E9432
:1062C0004C310C944B31DC01CB01FC01F999FECF30
:1062D00006C0F2BDE1BDF89A319600B40D9241506E
:0A62E0005040B8F70895F894FFCF7E
:1062EA0007000C52D02445000000410000DC4400A5
:1062FA0000004152D0A4440000404100005C440028
:10630A0000004148F17644000000415C978A44004D
:10631A000000411FD592440000004152D0A444001D
:10632A000000415CFFB844000000410AA7CF4400C6
:10633A000000410000DC44000000410AA7CF4400ED
:10634A000000410000DC44000000410000000000A1
:10635A0000804052D0244500004041000000000067
:10636A000080400AA74F45000040410AA7CF4400D9
:10637A000000410000DC4400000041000000000071
:10638A0000804052D0244500000041000000000077
:10639A000080405CFF38450000004100000000001A
:1063AA0000804052D02445000000410AA7CF440093
:1063BA000000410000DC4400000041000000000031
:1063CA0000804052D024450000804110F1764400FC
:1063DA0000A04112F1F6440000004141909B4400A4
:1063EA0000A04112F1F64400000041050000003F00
:1063FA000000C8426A14F814D514A1146D14016C73
:10640A00032808140A321E000002000400050007CF
:10641A000009000B000C000E0010001100130015FB
:10642A0000170018001A001C001D001F002100237D
:10643A000024002600280029002B002D002F003000
:10644A0000320034003500370039003B0042004575
:10645A000025002600430061006000200037006428
:10646A000065006600670044004600240047003FBC
:10647A004D36010BB40A7E0A2A0A430A5C0A010253
:08648A000304050607080900E0
:00000001FF
